Component: ARM Compiler 5.06 update 1 (build 61) Tool: armlink [4d35a8]

==============================================================================

Section Cross References

    startup_stm32f429_439xx.o(RESET) refers to startup_stm32f429_439xx.o(STACK) for __initial_sp
    startup_stm32f429_439xx.o(RESET) refers to startup_stm32f429_439xx.o(.text) for Reset_Handler
    startup_stm32f429_439xx.o(RESET) refers to stm32f4xx_it.o(.text) for NMI_Handler
    startup_stm32f429_439xx.o(RESET) refers to usb_bsp.o(.text) for OTG_HS_EP1_OUT_IRQHandler
    startup_stm32f429_439xx.o(.text) refers to system_stm32f4xx.o(.text) for SystemInit
    startup_stm32f429_439xx.o(.text) refers to entry.o(.ARM.Collect$$$$00000000) for __main
    stm32f4xx_rcc.o(.text) refers to stm32f4xx_rcc.o(.data) for .data
    stm32f4xx_gpio.o(.text) refers to stm32f4xx_rcc.o(.text) for RCC_AHB1PeriphResetCmd
    stm32f4xx_adc.o(.text) refers to stm32f4xx_rcc.o(.text) for RCC_APB2PeriphResetCmd
    stm32f4xx_tim.o(.text) refers to stm32f4xx_rcc.o(.text) for RCC_APB2PeriphResetCmd
    stm32f4xx_spi.o(.text) refers to stm32f4xx_rcc.o(.text) for RCC_APB1PeriphResetCmd
    stm32f4xx_dac.o(.text) refers to stm32f4xx_rcc.o(.text) for RCC_APB1PeriphResetCmd
    stm32f4xx_syscfg.o(.text) refers to stm32f4xx_rcc.o(.text) for RCC_APB2PeriphResetCmd
    stm32f4xx_fmc.o(.text) refers to stm32f4xx_fmc.o(.constdata) for .constdata
    tm_stm32f4_delay.o(.text) refers to stm32f4xx_rcc.o(.text) for RCC_HSEConfig
    tm_stm32f4_delay.o(.text) refers to tm_stm32f4_delay.o(.data) for .data
    tm_stm32f4_delay.o(.text) refers to system_stm32f4xx.o(.data) for SystemCoreClock
    tm_stm32f4_disco.o(.text) refers to stm32f4xx_rcc.o(.text) for RCC_AHB1PeriphClockCmd
    tm_stm32f4_disco.o(.text) refers to stm32f4xx_gpio.o(.text) for GPIO_Init
    tm_stm32f4_disco.o(.text) refers to tm_stm32f4_disco.o(.data) for .data
    tm_stm32f4_gpio.o(.text) refers to tm_stm32f4_gpio.o(.bss) for .bss
    tm_stm32f4_adc.o(.text) refers to stm32f4xx_adc.o(.text) for ADC_CommonInit
    tm_stm32f4_adc.o(.text) refers to tm_stm32f4_gpio.o(.text) for TM_GPIO_Init
    main.o(.text) refers to config.o(.text) for encoder1_config
    main.o(.text) refers to functions.o(.text) for escalado
    main.o(.text) refers to tm_stm32f4_delay.o(.text) for TM_DELAY_Init
    main.o(.text) refers to tm_stm32f4_disco.o(.text) for TM_DISCO_LedInit
    main.o(.text) refers to tm_stm32f4_sdram.o(.text) for TM_SDRAM_Init
    main.o(.text) refers to trapez.o(.text) for trapez4
    main.o(.text) refers to main.o(.bss) for .bss
    main.o(.text) refers to tm_stm32f4_delay.o(.data) for TM_Time
    stm32f4xx_it.o(.text) refers to tm_stm32f4_delay.o(.text) for TimingDelay_Decrement
    stm32f4xx_it.o(.text) refers to stm32f4xx_tim.o(.text) for TIM_GetITStatus
    stm32f4xx_it.o(.text) refers to stm32f4xx_exti.o(.text) for EXTI_GetITStatus
    stm32f4xx_it.o(.text) refers to paradaconrolada.o(.text) for paradacontrolada
    stm32f4xx_it.o(.text) refers to functions.o(.text) for escalado
    stm32f4xx_it.o(.text) refers to stm32f4xx_it.o(.data) for .data
    stm32f4xx_it.o(.text) refers to homing.o(.bss) for homing
    stm32f4xx_it.o(.text) refers to main.o(.bss) for encoder1
    system_stm32f4xx.o(.text) refers to system_stm32f4xx.o(.data) for .data
    tm_stm32f4_usb_vcp.o(.text) refers to usbd_core.o(.text) for USBD_Init
    tm_stm32f4_usb_vcp.o(.text) refers to usbd_cdc_vcp.o(.text) for VCP_DataTx
    tm_stm32f4_usb_vcp.o(.text) refers to usbd_usr.o(.data) for USR_cb
    tm_stm32f4_usb_vcp.o(.text) refers to usbd_cdc_core.o(.data) for USBD_CDC_cb
    tm_stm32f4_usb_vcp.o(.text) refers to usbd_desc.o(.data) for USR_desc
    tm_stm32f4_usb_vcp.o(.text) refers to tm_stm32f4_usb_vcp.o(.bss) for .bss
    tm_stm32f4_usb_vcp.o(.text) refers to tm_stm32f4_usb_vcp.o(.data) for .data
    tm_stm32f4_usb_vcp.o(.text) refers to usbd_usr.o(.data) for TM_USB_VCP_INT_Status
    tm_stm32f4_usb_vcp.o(.text) refers to usbd_cdc_vcp.o(.data) for linecoding
    tm_stm32f4_sdram.o(.text) refers to stm32f4xx_fmc.o(.text) for FMC_SDRAMInit
    tm_stm32f4_sdram.o(.text) refers to tm_stm32f4_gpio.o(.text) for TM_GPIO_InitAlternate
    tm_stm32f4_sdram.o(.text) refers to tm_stm32f4_sdram.o(.data) for .data
    config.o(.text) refers to stm32f4xx_rcc.o(.text) for RCC_APB1PeriphClockCmd
    config.o(.text) refers to stm32f4xx_tim.o(.text) for TIM_TimeBaseInit
    config.o(.text) refers to misc.o(.text) for NVIC_Init
    config.o(.text) refers to stm32f4xx_gpio.o(.text) for GPIO_Init
    config.o(.text) refers to stm32f4xx_dac.o(.text) for DAC_Init
    config.o(.text) refers to system_stm32f4xx.o(.data) for SystemCoreClock
    config.o(.text) refers to stm32f4xx_syscfg.o(.text) for SYSCFG_EXTILineConfig
    config.o(.text) refers to stm32f4xx_exti.o(.text) for EXTI_Init
    trapez.o(.text) refers to f2d.o(.text) for __aeabi_f2d
    trapez.o(.text) refers to ddiv.o(.text) for __aeabi_ddiv
    trapez.o(.text) refers to sqrt.o(i.__hardfp_sqrt) for __hardfp_sqrt
    trapez.o(.text) refers to d2f.o(.text) for __aeabi_d2f
    trapez.o(.text) refers to malloc.o(i.malloc) for malloc
    trapez.o(.text) refers to dmul.o(.text) for __aeabi_dmul
    trapez.o(.text) refers to dadd.o(.text) for __aeabi_dadd
    functions.o(.text) refers to f2d.o(.text) for __aeabi_f2d
    functions.o(.text) refers to dflti.o(.text) for __aeabi_i2d
    functions.o(.text) refers to dmul.o(.text) for __aeabi_dmul
    functions.o(.text) refers to ddiv.o(.text) for __aeabi_ddiv
    functions.o(.text) refers to d2f.o(.text) for __aeabi_d2f
    paradaconrolada.o(.text) refers to stm32f4xx_tim.o(.text) for TIM_ITConfig
    paradaconrolada.o(.text) refers to functions.o(.text) for vel_reference
    paradaconrolada.o(.text) refers to controller.o(.text) for PI_action
    paradaconrolada.o(.text) refers to paradaconrolada.o(.data) for .data
    paradaconrolada.o(.text) refers to main.o(.bss) for encoder3
    paradaconrolada.o(.text) refers to stm32f4xx_it.o(.data) for flag_Exp
    homing.o(.text) refers to functions.o(.text) for escalado
    homing.o(.text) refers to homing.o(.bss) for .bss
    homing.o(.text) refers to tm_stm32f4_delay.o(.data) for TM_Time
    usb_bsp.o(.text) refers to stm32f4xx_rcc.o(.text) for RCC_AHB1PeriphClockCmd
    usb_bsp.o(.text) refers to stm32f4xx_gpio.o(.text) for GPIO_Init
    usb_bsp.o(.text) refers to misc.o(.text) for NVIC_PriorityGroupConfig
    usb_bsp.o(.text) refers to stm32f4xx_exti.o(.text) for EXTI_ClearITPendingBit
    usb_bsp.o(.text) refers to usb_dcd_int.o(.text) for USBD_OTG_ISR_Handler
    usb_bsp.o(.text) refers to tm_stm32f4_usb_vcp.o(.bss) for USB_OTG_dev
    usb_core.o(.text) refers to usb_bsp.o(.text) for USB_OTG_BSP_uDelay
    usb_dcd.o(.text) refers to usb_core.o(.text) for USB_OTG_SelectCore
    usb_dcd.o(.text) refers to usb_bsp.o(.text) for USB_OTG_BSP_mDelay
    usb_dcd_int.o(.text) refers to usb_core.o(.text) for USB_OTG_WritePacket
    usb_dcd_int.o(.text) refers to usbd_core.o(.data) for USBD_DCD_INT_fops
    usbd_cdc_core.o(.text) refers to usb_dcd.o(.text) for DCD_EP_Open
    usbd_cdc_core.o(.text) refers to usbd_req.o(.text) for USBD_CtlError
    usbd_cdc_core.o(.text) refers to usbd_ioreq.o(.text) for USBD_CtlPrepareRx
    usbd_cdc_core.o(.text) refers to usbd_desc.o(.data) for USBD_DeviceDesc
    usbd_cdc_core.o(.text) refers to usbd_cdc_vcp.o(.data) for VCP_fops
    usbd_cdc_core.o(.text) refers to usbd_cdc_core.o(.bss) for .bss
    usbd_cdc_core.o(.text) refers to usbd_cdc_core.o(.data) for .data
    usbd_cdc_core.o(.data) refers to usbd_cdc_core.o(.text) for usbd_cdc_Init
    usbd_cdc_vcp.o(.text) refers to tm_stm32f4_usb_vcp.o(.text) for TM_INT_USB_VCP_AddReceived
    usbd_cdc_vcp.o(.text) refers to usbd_cdc_vcp.o(.data) for .data
    usbd_cdc_vcp.o(.text) refers to usbd_cdc_core.o(.data) for APP_Rx_ptr_in
    usbd_cdc_vcp.o(.text) refers to usbd_cdc_core.o(.bss) for APP_Rx_Buffer
    usbd_cdc_vcp.o(.data) refers to usbd_cdc_vcp.o(.text) for VCP_Init
    usbd_core.o(.text) refers to usb_bsp.o(.text) for USB_OTG_BSP_Init
    usbd_core.o(.text) refers to usb_dcd.o(.text) for DCD_Init
    usbd_core.o(.text) refers to usbd_req.o(.text) for USBD_ParseSetupRequest
    usbd_core.o(.text) refers to usbd_ioreq.o(.text) for USBD_CtlContinueRx
    usbd_core.o(.text) refers to usbd_core.o(.data) for .data
    usbd_core.o(.data) refers to usbd_core.o(.text) for USBD_DataOutStage
    usbd_core.o(.data) refers to usbd_core.o(.data) for USBD_DCD_INT_cb
    usbd_desc.o(.text) refers to usbd_req.o(.text) for USBD_GetString
    usbd_desc.o(.text) refers to usbd_desc.o(.data) for .data
    usbd_desc.o(.text) refers to usbd_req.o(.bss) for USBD_StrDesc
    usbd_desc.o(.data) refers to usbd_desc.o(.text) for USBD_USR_DeviceDescriptor
    usbd_ioreq.o(.text) refers to usb_dcd.o(.text) for DCD_EP_Tx
    usbd_ioreq.o(.text) refers to usb_core.o(.text) for USB_OTG_EP0_OutStart
    usbd_req.o(.text) refers to usb_dcd.o(.text) for DCD_EP_Stall
    usbd_req.o(.text) refers to usb_core.o(.text) for USB_OTG_EP0_OutStart
    usbd_req.o(.text) refers to usbd_core.o(.text) for USBD_ClrCfg
    usbd_req.o(.text) refers to usbd_ioreq.o(.text) for USBD_CtlSendStatus
    usbd_req.o(.text) refers to usbd_req.o(.data) for .data
    usbd_req.o(.text) refers to usbd_desc.o(.data) for USBD_DeviceQualifierDesc
    usbd_req.o(.text) refers to usbd_core.o(.data) for SET_TEST_MODE
    usbd_usr.o(.text) refers to usbd_usr.o(.data) for .data
    usbd_usr.o(.data) refers to usbd_usr.o(.text) for USBD_USR_Init
    sqrt.o(i.__hardfp_sqrt) refers (Special) to iusefp.o(.text) for __I$use$fp
    sqrt.o(i.__hardfp_sqrt) refers to dsqrt.o(.text) for _dsqrt
    sqrt.o(i.__hardfp_sqrt) refers to errno.o(i.__set_errno) for __set_errno
    sqrt.o(i.__softfp_sqrt) refers (Special) to iusefp.o(.text) for __I$use$fp
    sqrt.o(i.__softfp_sqrt) refers to dsqrt.o(.text) for _dsqrt
    sqrt.o(i.__softfp_sqrt) refers to errno.o(i.__set_errno) for __set_errno
    sqrt.o(i.sqrt) refers (Special) to iusefp.o(.text) for __I$use$fp
    sqrt.o(i.sqrt) refers to dsqrt.o(.text) for _dsqrt
    sqrt.o(i.sqrt) refers to errno.o(i.__set_errno) for __set_errno
    sqrt_x.o(i.____hardfp_sqrt$lsc) refers (Special) to iusefp.o(.text) for __I$use$fp
    sqrt_x.o(i.____hardfp_sqrt$lsc) refers to cdcmple.o(.text) for __aeabi_cdcmple
    sqrt_x.o(i.____hardfp_sqrt$lsc) refers to errno.o(i.__set_errno) for __set_errno
    sqrt_x.o(i.____hardfp_sqrt$lsc) refers to dsqrt.o(.text) for _dsqrt
    sqrt_x.o(i.____softfp_sqrt$lsc) refers (Special) to iusefp.o(.text) for __I$use$fp
    sqrt_x.o(i.____softfp_sqrt$lsc) refers to cdcmple.o(.text) for __aeabi_cdcmple
    sqrt_x.o(i.____softfp_sqrt$lsc) refers to errno.o(i.__set_errno) for __set_errno
    sqrt_x.o(i.____softfp_sqrt$lsc) refers to dsqrt.o(.text) for _dsqrt
    sqrt_x.o(i.__sqrt$lsc) refers (Special) to iusefp.o(.text) for __I$use$fp
    sqrt_x.o(i.__sqrt$lsc) refers to cdcmple.o(.text) for __aeabi_cdcmple
    sqrt_x.o(i.__sqrt$lsc) refers to errno.o(i.__set_errno) for __set_errno
    sqrt_x.o(i.__sqrt$lsc) refers to dsqrt.o(.text) for _dsqrt
    entry.o(.ARM.Collect$$$$00000000) refers (Special) to entry10a.o(.ARM.Collect$$$$0000000D) for __rt_final_cpp
    entry.o(.ARM.Collect$$$$00000000) refers (Special) to entry11a.o(.ARM.Collect$$$$0000000F) for __rt_final_exit
    entry.o(.ARM.Collect$$$$00000000) refers (Special) to entry7b.o(.ARM.Collect$$$$00000008) for _main_clock
    entry.o(.ARM.Collect$$$$00000000) refers (Special) to entry8b.o(.ARM.Collect$$$$0000000A) for _main_cpp_init
    entry.o(.ARM.Collect$$$$00000000) refers (Special) to entry9a.o(.ARM.Collect$$$$0000000B) for _main_init
    entry.o(.ARM.Collect$$$$00000000) refers (Special) to entry5.o(.ARM.Collect$$$$00000004) for _main_scatterload
    entry.o(.ARM.Collect$$$$00000000) refers (Special) to entry2.o(.ARM.Collect$$$$00000001) for _main_stk
    malloc.o(i.free) refers to mvars.o(.data) for __microlib_freelist
    malloc.o(i.malloc) refers to mvars.o(.data) for __microlib_freelist_initialised
    malloc.o(i.malloc) refers to mvars.o(.data) for __microlib_freelist
    malloc.o(i.malloc) refers to startup_stm32f429_439xx.o(HEAP) for __heap_base
    mallocr.o(i.__free$realloc) refers to mvars.o(.data) for __microlib_freelist
    mallocr.o(i.__malloc$realloc) refers to mallocr.o(i.internal_alloc) for internal_alloc
    mallocr.o(i.__malloc$realloc) refers to mvars.o(.data) for __microlib_freelist_initialised
    mallocr.o(i.__malloc$realloc) refers to startup_stm32f429_439xx.o(HEAP) for __heap_base
    mallocr.o(i.__malloc$realloc) refers to mvars.o(.data) for __microlib_freelist
    mallocr.o(i.internal_alloc) refers to memcpya.o(.text) for __aeabi_memcpy
    mallocr.o(i.internal_alloc) refers to mvars.o(.data) for __microlib_freelist
    mallocr.o(i.realloc) refers to mallocr.o(i.__free$realloc) for __free$realloc
    mallocr.o(i.realloc) refers to mallocr.o(i.internal_alloc) for internal_alloc
    mallocr.o(i.realloc) refers to mallocr.o(i.__malloc$realloc) for __malloc$realloc
    mallocr.o(i.realloc) refers to mvars.o(.data) for __microlib_freelist
    malloca.o(i.__aligned_malloc) refers to mvars.o(.data) for __microlib_freelist_initialised
    malloca.o(i.__aligned_malloc) refers to mvars.o(.data) for __microlib_freelist
    malloca.o(i.__aligned_malloc) refers to startup_stm32f429_439xx.o(HEAP) for __heap_base
    malloca.o(i.__free$memalign) refers to mvars.o(.data) for __microlib_freelist
    malloca.o(i.__malloc$memalign) refers to malloca.o(i.__aligned_malloc) for __aligned_malloc
    mallocra.o(i.__aligned_malloc$realloc) refers to mallocra.o(i.internal_alloc) for internal_alloc
    mallocra.o(i.__aligned_malloc$realloc) refers to mvars.o(.data) for __microlib_freelist_initialised
    mallocra.o(i.__aligned_malloc$realloc) refers to startup_stm32f429_439xx.o(HEAP) for __heap_base
    mallocra.o(i.__aligned_malloc$realloc) refers to mvars.o(.data) for __microlib_freelist
    mallocra.o(i.__free$realloc$memalign) refers to mvars.o(.data) for __microlib_freelist
    mallocra.o(i.__malloc$realloc$memalign) refers to mallocra.o(i.__aligned_malloc$realloc) for __aligned_malloc$realloc
    mallocra.o(i.__realloc$memalign) refers to mallocra.o(i.__free$realloc$memalign) for __free$realloc$memalign
    mallocra.o(i.__realloc$memalign) refers to mallocra.o(i.internal_alloc) for internal_alloc
    mallocra.o(i.__realloc$memalign) refers to mallocra.o(i.__malloc$realloc$memalign) for __malloc$realloc$memalign
    mallocra.o(i.__realloc$memalign) refers to mvars.o(.data) for __microlib_freelist
    mallocra.o(i.internal_alloc) refers to memcpya.o(.text) for __aeabi_memcpy
    mallocra.o(i.internal_alloc) refers to mvars.o(.data) for __microlib_freelist
    dadd.o(.text) refers (Special) to iusefp.o(.text) for __I$use$fp
    dadd.o(.text) refers to llshl.o(.text) for __aeabi_llsl
    dadd.o(.text) refers to llsshr.o(.text) for __aeabi_lasr
    dadd.o(.text) refers to depilogue.o(.text) for _double_epilogue
    dmul.o(.text) refers (Special) to iusefp.o(.text) for __I$use$fp
    dmul.o(.text) refers to depilogue.o(.text) for _double_epilogue
    ddiv.o(.text) refers (Special) to iusefp.o(.text) for __I$use$fp
    ddiv.o(.text) refers to depilogue.o(.text) for _double_round
    dflti.o(.text) refers (Special) to iusefp.o(.text) for __I$use$fp
    dflti.o(.text) refers to depilogue.o(.text) for _double_epilogue
    f2d.o(.text) refers (Special) to iusefp.o(.text) for __I$use$fp
    d2f.o(.text) refers (Special) to iusefp.o(.text) for __I$use$fp
    d2f.o(.text) refers to fepilogue.o(.text) for _float_round
    entry2.o(.ARM.Collect$$$$00000001) refers to entry2.o(.ARM.Collect$$$$00002712) for __lit__00000000
    entry2.o(.ARM.Collect$$$$00002712) refers to startup_stm32f429_439xx.o(STACK) for __initial_sp
    entry2.o(__vectab_stack_and_reset_area) refers to startup_stm32f429_439xx.o(STACK) for __initial_sp
    entry2.o(__vectab_stack_and_reset_area) refers to entry.o(.ARM.Collect$$$$00000000) for __main
    entry5.o(.ARM.Collect$$$$00000004) refers to init.o(.text) for __scatterload
    entry9a.o(.ARM.Collect$$$$0000000B) refers to main.o(.text) for main
    entry9b.o(.ARM.Collect$$$$0000000C) refers to main.o(.text) for main
    errno.o(i.__aeabi_errno_addr) refers to errno.o(.data) for .data
    errno.o(i.__read_errno) refers to errno.o(.data) for .data
    errno.o(i.__set_errno) refers to errno.o(.data) for .data
    depilogue.o(.text) refers to llshl.o(.text) for __aeabi_llsl
    depilogue.o(.text) refers to llushr.o(.text) for __aeabi_llsr
    dsqrt.o(.text) refers to llushr.o(.text) for __aeabi_llsr
    dsqrt.o(.text) refers to depilogue.o(.text) for _double_round
    init.o(.text) refers to entry5.o(.ARM.Collect$$$$00000004) for __main_after_scatterload


==============================================================================

Removing Unused input sections from the image.

    Removing misc.o(.rev16_text), (4 bytes).
    Removing misc.o(.revsh_text), (4 bytes).
    Removing misc.o(.rrx_text), (6 bytes).
    Removing stm32f4xx_rcc.o(.rev16_text), (4 bytes).
    Removing stm32f4xx_rcc.o(.revsh_text), (4 bytes).
    Removing stm32f4xx_rcc.o(.rrx_text), (6 bytes).
    Removing stm32f4xx_gpio.o(.rev16_text), (4 bytes).
    Removing stm32f4xx_gpio.o(.revsh_text), (4 bytes).
    Removing stm32f4xx_gpio.o(.rrx_text), (6 bytes).
    Removing stm32f4xx_adc.o(.rev16_text), (4 bytes).
    Removing stm32f4xx_adc.o(.revsh_text), (4 bytes).
    Removing stm32f4xx_adc.o(.rrx_text), (6 bytes).
    Removing stm32f4xx_adc.o(.text), (852 bytes).
    Removing stm32f4xx_exti.o(.rev16_text), (4 bytes).
    Removing stm32f4xx_exti.o(.revsh_text), (4 bytes).
    Removing stm32f4xx_exti.o(.rrx_text), (6 bytes).
    Removing stm32f4xx_tim.o(.rev16_text), (4 bytes).
    Removing stm32f4xx_tim.o(.revsh_text), (4 bytes).
    Removing stm32f4xx_tim.o(.rrx_text), (6 bytes).
    Removing stm32f4xx_spi.o(.rev16_text), (4 bytes).
    Removing stm32f4xx_spi.o(.revsh_text), (4 bytes).
    Removing stm32f4xx_spi.o(.rrx_text), (6 bytes).
    Removing stm32f4xx_spi.o(.text), (812 bytes).
    Removing stm32f4xx_dac.o(.rev16_text), (4 bytes).
    Removing stm32f4xx_dac.o(.revsh_text), (4 bytes).
    Removing stm32f4xx_dac.o(.rrx_text), (6 bytes).
    Removing stm32f4xx_dma.o(.rev16_text), (4 bytes).
    Removing stm32f4xx_dma.o(.revsh_text), (4 bytes).
    Removing stm32f4xx_dma.o(.rrx_text), (6 bytes).
    Removing stm32f4xx_dma.o(.text), (800 bytes).
    Removing stm32f4xx_syscfg.o(.rev16_text), (4 bytes).
    Removing stm32f4xx_syscfg.o(.revsh_text), (4 bytes).
    Removing stm32f4xx_syscfg.o(.rrx_text), (6 bytes).
    Removing stm32f4xx_fmc.o(.rev16_text), (4 bytes).
    Removing stm32f4xx_fmc.o(.revsh_text), (4 bytes).
    Removing stm32f4xx_fmc.o(.rrx_text), (6 bytes).
    Removing tm_stm32f4_delay.o(.rev16_text), (4 bytes).
    Removing tm_stm32f4_delay.o(.revsh_text), (4 bytes).
    Removing tm_stm32f4_delay.o(.rrx_text), (6 bytes).
    Removing tm_stm32f4_delay.o(.data), (4 bytes).
    Removing tm_stm32f4_disco.o(.rev16_text), (4 bytes).
    Removing tm_stm32f4_disco.o(.revsh_text), (4 bytes).
    Removing tm_stm32f4_disco.o(.rrx_text), (6 bytes).
    Removing tm_stm32f4_gpio.o(.rev16_text), (4 bytes).
    Removing tm_stm32f4_gpio.o(.revsh_text), (4 bytes).
    Removing tm_stm32f4_gpio.o(.rrx_text), (6 bytes).
    Removing tm_stm32f4_adc.o(.rev16_text), (4 bytes).
    Removing tm_stm32f4_adc.o(.revsh_text), (4 bytes).
    Removing tm_stm32f4_adc.o(.rrx_text), (6 bytes).
    Removing tm_stm32f4_adc.o(.text), (828 bytes).
    Removing tm_stm32f4_rng.o(.rev16_text), (4 bytes).
    Removing tm_stm32f4_rng.o(.revsh_text), (4 bytes).
    Removing tm_stm32f4_rng.o(.rrx_text), (6 bytes).
    Removing tm_stm32f4_rng.o(.text), (72 bytes).
    Removing main.o(.rev16_text), (4 bytes).
    Removing main.o(.revsh_text), (4 bytes).
    Removing main.o(.rrx_text), (6 bytes).
    Removing main.o(.bss), (22272 bytes).
    Removing main.o(.bss), (22272 bytes).
    Removing main.o(.bss), (11168 bytes).
    Removing main.o(.data), (4 bytes).
    Removing main.o(.data), (4 bytes).
    Removing main.o(.data), (4 bytes).
    Removing main.o(.data), (4 bytes).
    Removing main.o(.data), (4 bytes).
    Removing main.o(.data), (4 bytes).
    Removing main.o(.data), (4 bytes).
    Removing main.o(.data), (4 bytes).
    Removing main.o(.data), (4 bytes).
    Removing main.o(.data), (4 bytes).
    Removing main.o(.data), (4 bytes).
    Removing main.o(.data), (4 bytes).
    Removing main.o(.data), (4 bytes).
    Removing main.o(.data), (4 bytes).
    Removing main.o(.data), (4 bytes).
    Removing main.o(.data), (4 bytes).
    Removing main.o(.data), (4 bytes).
    Removing main.o(.data), (16 bytes).
    Removing stm32f4xx_it.o(.rev16_text), (4 bytes).
    Removing stm32f4xx_it.o(.revsh_text), (4 bytes).
    Removing stm32f4xx_it.o(.rrx_text), (6 bytes).
    Removing system_stm32f4xx.o(.rev16_text), (4 bytes).
    Removing system_stm32f4xx.o(.revsh_text), (4 bytes).
    Removing system_stm32f4xx.o(.rrx_text), (6 bytes).
    Removing tm_stm32f4_usb_vcp.o(.rev16_text), (4 bytes).
    Removing tm_stm32f4_usb_vcp.o(.revsh_text), (4 bytes).
    Removing tm_stm32f4_usb_vcp.o(.rrx_text), (6 bytes).
    Removing tm_stm32f4_usb_vcp.o(.text), (412 bytes).
    Removing tm_stm32f4_usb_vcp.o(.data), (16 bytes).
    Removing tm_stm32f4_sdram.o(.rev16_text), (4 bytes).
    Removing tm_stm32f4_sdram.o(.revsh_text), (4 bytes).
    Removing tm_stm32f4_sdram.o(.rrx_text), (6 bytes).
    Removing config.o(.rev16_text), (4 bytes).
    Removing config.o(.revsh_text), (4 bytes).
    Removing config.o(.rrx_text), (6 bytes).
    Removing trapez.o(.rev16_text), (4 bytes).
    Removing trapez.o(.revsh_text), (4 bytes).
    Removing trapez.o(.rrx_text), (6 bytes).
    Removing paradaconrolada.o(.rev16_text), (4 bytes).
    Removing paradaconrolada.o(.revsh_text), (4 bytes).
    Removing paradaconrolada.o(.rrx_text), (6 bytes).
    Removing paradaconrolada.o(.data), (4 bytes).
    Removing paradaconrolada.o(.data), (4 bytes).
    Removing homing.o(.rev16_text), (4 bytes).
    Removing homing.o(.revsh_text), (4 bytes).
    Removing homing.o(.rrx_text), (6 bytes).
    Removing homing.o(.text), (332 bytes).
    Removing usb_bsp.o(.rev16_text), (4 bytes).
    Removing usb_bsp.o(.revsh_text), (4 bytes).
    Removing usb_bsp.o(.rrx_text), (6 bytes).
    Removing usb_core.o(.rev16_text), (4 bytes).
    Removing usb_core.o(.revsh_text), (4 bytes).
    Removing usb_core.o(.rrx_text), (6 bytes).
    Removing usb_dcd.o(.rev16_text), (4 bytes).
    Removing usb_dcd.o(.revsh_text), (4 bytes).
    Removing usb_dcd.o(.rrx_text), (6 bytes).
    Removing usb_dcd_int.o(.rev16_text), (4 bytes).
    Removing usb_dcd_int.o(.revsh_text), (4 bytes).
    Removing usb_dcd_int.o(.rrx_text), (6 bytes).
    Removing usbd_cdc_core.o(.rev16_text), (4 bytes).
    Removing usbd_cdc_core.o(.revsh_text), (4 bytes).
    Removing usbd_cdc_core.o(.rrx_text), (6 bytes).
    Removing usbd_cdc_core.o(.text), (584 bytes).
    Removing usbd_cdc_core.o(.bss), (2112 bytes).
    Removing usbd_cdc_core.o(.data), (174 bytes).
    Removing usbd_cdc_core.o(.data), (48 bytes).
    Removing usbd_cdc_vcp.o(.rev16_text), (4 bytes).
    Removing usbd_cdc_vcp.o(.revsh_text), (4 bytes).
    Removing usbd_cdc_vcp.o(.rrx_text), (6 bytes).
    Removing usbd_cdc_vcp.o(.text), (172 bytes).
    Removing usbd_cdc_vcp.o(.data), (8 bytes).
    Removing usbd_cdc_vcp.o(.data), (20 bytes).
    Removing usbd_core.o(.rev16_text), (4 bytes).
    Removing usbd_core.o(.revsh_text), (4 bytes).
    Removing usbd_core.o(.rrx_text), (6 bytes).
    Removing usbd_desc.o(.rev16_text), (4 bytes).
    Removing usbd_desc.o(.revsh_text), (4 bytes).
    Removing usbd_desc.o(.rrx_text), (6 bytes).
    Removing usbd_desc.o(.text), (208 bytes).
    Removing usbd_desc.o(.data), (28 bytes).
    Removing usbd_desc.o(.data), (22 bytes).
    Removing usbd_ioreq.o(.rev16_text), (4 bytes).
    Removing usbd_ioreq.o(.revsh_text), (4 bytes).
    Removing usbd_ioreq.o(.rrx_text), (6 bytes).
    Removing usbd_req.o(.rev16_text), (4 bytes).
    Removing usbd_req.o(.revsh_text), (4 bytes).
    Removing usbd_req.o(.rrx_text), (6 bytes).
    Removing usbd_req.o(.bss), (255 bytes).
    Removing usbd_usr.o(.rev16_text), (4 bytes).
    Removing usbd_usr.o(.revsh_text), (4 bytes).
    Removing usbd_usr.o(.rrx_text), (6 bytes).
    Removing usbd_usr.o(.text), (68 bytes).
    Removing usbd_usr.o(.data), (1 bytes).
    Removing usbd_usr.o(.data), (28 bytes).
    Removing cdcmple.o(.text), (48 bytes).

155 unused section(s) (total 64212 bytes) removed from the image.

==============================================================================

Image Symbol Table

    Local Symbols

    Symbol Name                              Value     Ov Type        Size  Object(Section)

    ../clib/microlib/errno.c                 0x00000000   Number         0  errno.o ABSOLUTE
    ../clib/microlib/init/entry.s            0x00000000   Number         0  entry5.o ABSOLUTE
    ../clib/microlib/init/entry.s            0x00000000   Number         0  entry.o ABSOLUTE
    ../clib/microlib/init/entry.s            0x00000000   Number         0  entry7a.o ABSOLUTE
    ../clib/microlib/init/entry.s            0x00000000   Number         0  entry8b.o ABSOLUTE
    ../clib/microlib/init/entry.s            0x00000000   Number         0  entry7b.o ABSOLUTE
    ../clib/microlib/init/entry.s            0x00000000   Number         0  entry8a.o ABSOLUTE
    ../clib/microlib/init/entry.s            0x00000000   Number         0  entry9a.o ABSOLUTE
    ../clib/microlib/init/entry.s            0x00000000   Number         0  entry10a.o ABSOLUTE
    ../clib/microlib/init/entry.s            0x00000000   Number         0  entry10b.o ABSOLUTE
    ../clib/microlib/init/entry.s            0x00000000   Number         0  entry11b.o ABSOLUTE
    ../clib/microlib/init/entry.s            0x00000000   Number         0  entry11a.o ABSOLUTE
    ../clib/microlib/init/entry.s            0x00000000   Number         0  entry2.o ABSOLUTE
    ../clib/microlib/init/entry.s            0x00000000   Number         0  entry9b.o ABSOLUTE
    ../clib/microlib/longlong.c              0x00000000   Number         0  llushr.o ABSOLUTE
    ../clib/microlib/longlong.c              0x00000000   Number         0  llsshr.o ABSOLUTE
    ../clib/microlib/longlong.c              0x00000000   Number         0  llshl.o ABSOLUTE
    ../clib/microlib/malloc/malloc.c         0x00000000   Number         0  mallocr.o ABSOLUTE
    ../clib/microlib/malloc/malloc.c         0x00000000   Number         0  malloc.o ABSOLUTE
    ../clib/microlib/malloc/malloc.c         0x00000000   Number         0  malloca.o ABSOLUTE
    ../clib/microlib/malloc/malloc.c         0x00000000   Number         0  mallocra.o ABSOLUTE
    ../clib/microlib/malloc/mvars.c          0x00000000   Number         0  mvars.o ABSOLUTE
    ../clib/microlib/string/memcpy.c         0x00000000   Number         0  memcpya.o ABSOLUTE
    ../clib/microlib/string/memcpy.c         0x00000000   Number         0  memcpyb.o ABSOLUTE
    ../clib/microlib/stubs.s                 0x00000000   Number         0  iusefp.o ABSOLUTE
    ../fplib/microlib/d2f.c                  0x00000000   Number         0  d2f.o ABSOLUTE
    ../fplib/microlib/f2d.c                  0x00000000   Number         0  f2d.o ABSOLUTE
    ../fplib/microlib/fpadd.c                0x00000000   Number         0  dadd.o ABSOLUTE
    ../fplib/microlib/fpdiv.c                0x00000000   Number         0  ddiv.o ABSOLUTE
    ../fplib/microlib/fpepilogue.c           0x00000000   Number         0  fepilogue.o ABSOLUTE
    ../fplib/microlib/fpepilogue.c           0x00000000   Number         0  depilogue.o ABSOLUTE
    ../fplib/microlib/fpflt.c                0x00000000   Number         0  dflti.o ABSOLUTE
    ../fplib/microlib/fpmul.c                0x00000000   Number         0  dmul.o ABSOLUTE
    ../fplib/microlib/fpsqrt.c               0x00000000   Number         0  dsqrt.o ABSOLUTE
    ../mathlib/sqrt.c                        0x00000000   Number         0  sqrt_x.o ABSOLUTE
    ../mathlib/sqrt.c                        0x00000000   Number         0  sqrt.o ABSOLUTE
    ..\00-STM32F429_LIBRARIES\tm_stm32f4_delay.c 0x00000000   Number         0  tm_stm32f4_delay.o ABSOLUTE
    ..\00-STM32F429_LIBRARIES\tm_stm32f4_disco.c 0x00000000   Number         0  tm_stm32f4_disco.o ABSOLUTE
    ..\00-STM32F429_LIBRARIES\tm_stm32f4_gpio.c 0x00000000   Number         0  tm_stm32f4_gpio.o ABSOLUTE
    ..\00-STM32F4xx_STANDARD_PERIPHERAL_DRIVERS\CMSIS\Device\ST\STM32F4xx\Source\Templates\arm\startup_stm32f429_439xx.s 0x00000000   Number         0  startup_stm32f429_439xx.o ABSOLUTE
    ..\00-STM32F4xx_STANDARD_PERIPHERAL_DRIVERS\STM32F4xx_StdPeriph_Driver\src\misc.c 0x00000000   Number         0  misc.o ABSOLUTE
    ..\00-STM32F4xx_STANDARD_PERIPHERAL_DRIVERS\STM32F4xx_StdPeriph_Driver\src\stm32f4xx_adc.c 0x00000000   Number         0  stm32f4xx_adc.o ABSOLUTE
    ..\00-STM32F4xx_STANDARD_PERIPHERAL_DRIVERS\STM32F4xx_StdPeriph_Driver\src\stm32f4xx_dac.c 0x00000000   Number         0  stm32f4xx_dac.o ABSOLUTE
    ..\00-STM32F4xx_STANDARD_PERIPHERAL_DRIVERS\STM32F4xx_StdPeriph_Driver\src\stm32f4xx_dma.c 0x00000000   Number         0  stm32f4xx_dma.o ABSOLUTE
    ..\00-STM32F4xx_STANDARD_PERIPHERAL_DRIVERS\STM32F4xx_StdPeriph_Driver\src\stm32f4xx_exti.c 0x00000000   Number         0  stm32f4xx_exti.o ABSOLUTE
    ..\00-STM32F4xx_STANDARD_PERIPHERAL_DRIVERS\STM32F4xx_StdPeriph_Driver\src\stm32f4xx_fmc.c 0x00000000   Number         0  stm32f4xx_fmc.o ABSOLUTE
    ..\00-STM32F4xx_STANDARD_PERIPHERAL_DRIVERS\STM32F4xx_StdPeriph_Driver\src\stm32f4xx_gpio.c 0x00000000   Number         0  stm32f4xx_gpio.o ABSOLUTE
    ..\00-STM32F4xx_STANDARD_PERIPHERAL_DRIVERS\STM32F4xx_StdPeriph_Driver\src\stm32f4xx_rcc.c 0x00000000   Number         0  stm32f4xx_rcc.o ABSOLUTE
    ..\00-STM32F4xx_STANDARD_PERIPHERAL_DRIVERS\STM32F4xx_StdPeriph_Driver\src\stm32f4xx_spi.c 0x00000000   Number         0  stm32f4xx_spi.o ABSOLUTE
    ..\00-STM32F4xx_STANDARD_PERIPHERAL_DRIVERS\STM32F4xx_StdPeriph_Driver\src\stm32f4xx_syscfg.c 0x00000000   Number         0  stm32f4xx_syscfg.o ABSOLUTE
    ..\00-STM32F4xx_STANDARD_PERIPHERAL_DRIVERS\STM32F4xx_StdPeriph_Driver\src\stm32f4xx_tim.c 0x00000000   Number         0  stm32f4xx_tim.o ABSOLUTE
    ..\\00-STM32F429_LIBRARIES\\tm_stm32f4_delay.c 0x00000000   Number         0  tm_stm32f4_delay.o ABSOLUTE
    ..\\00-STM32F429_LIBRARIES\\tm_stm32f4_disco.c 0x00000000   Number         0  tm_stm32f4_disco.o ABSOLUTE
    ..\\00-STM32F429_LIBRARIES\\tm_stm32f4_gpio.c 0x00000000   Number         0  tm_stm32f4_gpio.o ABSOLUTE
    ..\\00-STM32F4xx_STANDARD_PERIPHERAL_DRIVERS\\STM32F4xx_StdPeriph_Driver\\src\\misc.c 0x00000000   Number         0  misc.o ABSOLUTE
    ..\\00-STM32F4xx_STANDARD_PERIPHERAL_DRIVERS\\STM32F4xx_StdPeriph_Driver\\src\\stm32f4xx_adc.c 0x00000000   Number         0  stm32f4xx_adc.o ABSOLUTE
    ..\\00-STM32F4xx_STANDARD_PERIPHERAL_DRIVERS\\STM32F4xx_StdPeriph_Driver\\src\\stm32f4xx_dac.c 0x00000000   Number         0  stm32f4xx_dac.o ABSOLUTE
    ..\\00-STM32F4xx_STANDARD_PERIPHERAL_DRIVERS\\STM32F4xx_StdPeriph_Driver\\src\\stm32f4xx_dma.c 0x00000000   Number         0  stm32f4xx_dma.o ABSOLUTE
    ..\\00-STM32F4xx_STANDARD_PERIPHERAL_DRIVERS\\STM32F4xx_StdPeriph_Driver\\src\\stm32f4xx_exti.c 0x00000000   Number         0  stm32f4xx_exti.o ABSOLUTE
    ..\\00-STM32F4xx_STANDARD_PERIPHERAL_DRIVERS\\STM32F4xx_StdPeriph_Driver\\src\\stm32f4xx_fmc.c 0x00000000   Number         0  stm32f4xx_fmc.o ABSOLUTE
    ..\\00-STM32F4xx_STANDARD_PERIPHERAL_DRIVERS\\STM32F4xx_StdPeriph_Driver\\src\\stm32f4xx_gpio.c 0x00000000   Number         0  stm32f4xx_gpio.o ABSOLUTE
    ..\\00-STM32F4xx_STANDARD_PERIPHERAL_DRIVERS\\STM32F4xx_StdPeriph_Driver\\src\\stm32f4xx_rcc.c 0x00000000   Number         0  stm32f4xx_rcc.o ABSOLUTE
    ..\\00-STM32F4xx_STANDARD_PERIPHERAL_DRIVERS\\STM32F4xx_StdPeriph_Driver\\src\\stm32f4xx_spi.c 0x00000000   Number         0  stm32f4xx_spi.o ABSOLUTE
    ..\\00-STM32F4xx_STANDARD_PERIPHERAL_DRIVERS\\STM32F4xx_StdPeriph_Driver\\src\\stm32f4xx_syscfg.c 0x00000000   Number         0  stm32f4xx_syscfg.o ABSOLUTE
    ..\\00-STM32F4xx_STANDARD_PERIPHERAL_DRIVERS\\STM32F4xx_StdPeriph_Driver\\src\\stm32f4xx_tim.c 0x00000000   Number         0  stm32f4xx_tim.o ABSOLUTE
    User\\config.c                           0x00000000   Number         0  config.o ABSOLUTE
    User\\homing.c                           0x00000000   Number         0  homing.o ABSOLUTE
    User\\main.c                             0x00000000   Number         0  main.o ABSOLUTE
    User\\paradaconrolada.c                  0x00000000   Number         0  paradaconrolada.o ABSOLUTE
    User\\stm32f4xx_it.c                     0x00000000   Number         0  stm32f4xx_it.o ABSOLUTE
    User\\system_stm32f4xx.c                 0x00000000   Number         0  system_stm32f4xx.o ABSOLUTE
    User\\tm_stm32f4_adc.c                   0x00000000   Number         0  tm_stm32f4_adc.o ABSOLUTE
    User\\tm_stm32f4_rng.c                   0x00000000   Number         0  tm_stm32f4_rng.o ABSOLUTE
    User\\tm_stm32f4_sdram.c                 0x00000000   Number         0  tm_stm32f4_sdram.o ABSOLUTE
    User\\tm_stm32f4_usb_vcp.c               0x00000000   Number         0  tm_stm32f4_usb_vcp.o ABSOLUTE
    User\\trapez.c                           0x00000000   Number         0  trapez.o ABSOLUTE
    User\\usb_bsp.c                          0x00000000   Number         0  usb_bsp.o ABSOLUTE
    User\\usb_core.c                         0x00000000   Number         0  usb_core.o ABSOLUTE
    User\\usb_dcd.c                          0x00000000   Number         0  usb_dcd.o ABSOLUTE
    User\\usb_dcd_int.c                      0x00000000   Number         0  usb_dcd_int.o ABSOLUTE
    User\\usbd_cdc_core.c                    0x00000000   Number         0  usbd_cdc_core.o ABSOLUTE
    User\\usbd_cdc_vcp.c                     0x00000000   Number         0  usbd_cdc_vcp.o ABSOLUTE
    User\\usbd_core.c                        0x00000000   Number         0  usbd_core.o ABSOLUTE
    User\\usbd_desc.c                        0x00000000   Number         0  usbd_desc.o ABSOLUTE
    User\\usbd_ioreq.c                       0x00000000   Number         0  usbd_ioreq.o ABSOLUTE
    User\\usbd_req.c                         0x00000000   Number         0  usbd_req.o ABSOLUTE
    User\\usbd_usr.c                         0x00000000   Number         0  usbd_usr.o ABSOLUTE
    User\config.c                            0x00000000   Number         0  config.o ABSOLUTE
    User\controller.c                        0x00000000   Number         0  controller.o ABSOLUTE
    User\functions.c                         0x00000000   Number         0  functions.o ABSOLUTE
    User\homing.c                            0x00000000   Number         0  homing.o ABSOLUTE
    User\main.c                              0x00000000   Number         0  main.o ABSOLUTE
    User\paradaconrolada.c                   0x00000000   Number         0  paradaconrolada.o ABSOLUTE
    User\stm32f4xx_it.c                      0x00000000   Number         0  stm32f4xx_it.o ABSOLUTE
    User\system_stm32f4xx.c                  0x00000000   Number         0  system_stm32f4xx.o ABSOLUTE
    User\tm_stm32f4_adc.c                    0x00000000   Number         0  tm_stm32f4_adc.o ABSOLUTE
    User\tm_stm32f4_rng.c                    0x00000000   Number         0  tm_stm32f4_rng.o ABSOLUTE
    User\tm_stm32f4_sdram.c                  0x00000000   Number         0  tm_stm32f4_sdram.o ABSOLUTE
    User\tm_stm32f4_usb_vcp.c                0x00000000   Number         0  tm_stm32f4_usb_vcp.o ABSOLUTE
    User\trapez.c                            0x00000000   Number         0  trapez.o ABSOLUTE
    User\usb_bsp.c                           0x00000000   Number         0  usb_bsp.o ABSOLUTE
    User\usb_core.c                          0x00000000   Number         0  usb_core.o ABSOLUTE
    User\usb_dcd.c                           0x00000000   Number         0  usb_dcd.o ABSOLUTE
    User\usb_dcd_int.c                       0x00000000   Number         0  usb_dcd_int.o ABSOLUTE
    User\usbd_cdc_core.c                     0x00000000   Number         0  usbd_cdc_core.o ABSOLUTE
    User\usbd_cdc_vcp.c                      0x00000000   Number         0  usbd_cdc_vcp.o ABSOLUTE
    User\usbd_core.c                         0x00000000   Number         0  usbd_core.o ABSOLUTE
    User\usbd_desc.c                         0x00000000   Number         0  usbd_desc.o ABSOLUTE
    User\usbd_ioreq.c                        0x00000000   Number         0  usbd_ioreq.o ABSOLUTE
    User\usbd_req.c                          0x00000000   Number         0  usbd_req.o ABSOLUTE
    User\usbd_usr.c                          0x00000000   Number         0  usbd_usr.o ABSOLUTE
    cdcmple.s                                0x00000000   Number         0  cdcmple.o ABSOLUTE
    dc.s                                     0x00000000   Number         0  dc.o ABSOLUTE
    handlers.s                               0x00000000   Number         0  handlers.o ABSOLUTE
    init.s                                   0x00000000   Number         0  init.o ABSOLUTE
    RESET                                    0x08000000   Section      428  startup_stm32f429_439xx.o(RESET)
    .ARM.Collect$$$$00000000                 0x080001ac   Section        0  entry.o(.ARM.Collect$$$$00000000)
    .ARM.Collect$$$$00000001                 0x080001ac   Section        4  entry2.o(.ARM.Collect$$$$00000001)
    .ARM.Collect$$$$00000004                 0x080001b0   Section        4  entry5.o(.ARM.Collect$$$$00000004)
    .ARM.Collect$$$$00000008                 0x080001b4   Section        0  entry7b.o(.ARM.Collect$$$$00000008)
    .ARM.Collect$$$$0000000A                 0x080001b4   Section        0  entry8b.o(.ARM.Collect$$$$0000000A)
    .ARM.Collect$$$$0000000B                 0x080001b4   Section        8  entry9a.o(.ARM.Collect$$$$0000000B)
    .ARM.Collect$$$$0000000D                 0x080001bc   Section        0  entry10a.o(.ARM.Collect$$$$0000000D)
    .ARM.Collect$$$$0000000F                 0x080001bc   Section        0  entry11a.o(.ARM.Collect$$$$0000000F)
    .ARM.Collect$$$$00002712                 0x080001bc   Section        4  entry2.o(.ARM.Collect$$$$00002712)
    __lit__00000000                          0x080001bc   Data           4  entry2.o(.ARM.Collect$$$$00002712)
    .text                                    0x080001c0   Section       36  startup_stm32f429_439xx.o(.text)
    $v0                                      0x080001c0   Number         0  startup_stm32f429_439xx.o(.text)
    .text                                    0x080001e4   Section        0  misc.o(.text)
    .text                                    0x08000294   Section        0  stm32f4xx_rcc.o(.text)
    .text                                    0x08000718   Section        0  stm32f4xx_gpio.o(.text)
    .text                                    0x08000924   Section        0  stm32f4xx_exti.o(.text)
    .text                                    0x08000a04   Section        0  stm32f4xx_tim.o(.text)
    TI2_Config                               0x0800104f   Thumb Code    54  stm32f4xx_tim.o(.text)
    TI1_Config                               0x080013b3   Thumb Code    46  stm32f4xx_tim.o(.text)
    .text                                    0x080013e0   Section        0  stm32f4xx_dac.o(.text)
    .text                                    0x08001534   Section        0  stm32f4xx_syscfg.o(.text)
    .text                                    0x080015b0   Section        0  stm32f4xx_fmc.o(.text)
    .text                                    0x08001d08   Section        0  tm_stm32f4_delay.o(.text)
    .text                                    0x08001da8   Section        0  tm_stm32f4_disco.o(.text)
    .text                                    0x08001e44   Section        0  tm_stm32f4_gpio.o(.text)
    .text                                    0x080020e0   Section        0  main.o(.text)
    NVIC_EnableIRQ                           0x080021d5   Thumb Code    22  main.o(.text)
    .text                                    0x08002208   Section        0  stm32f4xx_it.o(.text)
    .text                                    0x08002398   Section        0  system_stm32f4xx.o(.text)
    SetSysClock                              0x08002399   Thumb Code   190  system_stm32f4xx.o(.text)
    .text                                    0x08002530   Section        0  tm_stm32f4_sdram.o(.text)
    TM_SDRAM_InitPins                        0x080026a5   Thumb Code   120  tm_stm32f4_sdram.o(.text)
    .text                                    0x08002740   Section        0  config.o(.text)
    .text                                    0x08002cf8   Section        0  trapez.o(.text)
    .text                                    0x08003868   Section        0  functions.o(.text)
    .text                                    0x08003964   Section        0  controller.o(.text)
    .text                                    0x080039c0   Section        0  paradaconrolada.o(.text)
    .text                                    0x08003ae8   Section        0  usb_bsp.o(.text)
    .text                                    0x08003c3c   Section        0  usb_core.o(.text)
    USB_OTG_CoreReset                        0x08003c3d   Thumb Code    84  usb_core.o(.text)
    .text                                    0x080045c4   Section        0  usb_dcd.o(.text)
    .text                                    0x08004844   Section        0  usb_dcd_int.o(.text)
    DCD_WriteEmptyTxFifo                     0x0800488f   Thumb Code   114  usb_dcd_int.o(.text)
    DCD_HandleInEP_ISR                       0x08004975   Thumb Code   198  usb_dcd_int.o(.text)
    DCD_HandleUsbReset_ISR                   0x08004b7f   Thumb Code   138  usb_dcd_int.o(.text)
    DCD_HandleRxStatusQueueLevel_ISR         0x08004c09   Thumb Code   128  usb_dcd_int.o(.text)
    DCD_HandleUSBSuspend_ISR                 0x08004c89   Thumb Code   102  usb_dcd_int.o(.text)
    DCD_HandleOutEP_ISR                      0x08004cef   Thumb Code   164  usb_dcd_int.o(.text)
    .text                                    0x08004d9c   Section        0  usbd_core.o(.text)
    USBD_SetupStage                          0x08004dd5   Thumb Code    72  usbd_core.o(.text)
    USBD_DataOutStage                        0x08004e1d   Thumb Code   116  usbd_core.o(.text)
    USBD_DataInStage                         0x08004e91   Thumb Code   172  usbd_core.o(.text)
    USBD_Reset                               0x08004f3d   Thumb Code    46  usbd_core.o(.text)
    USBD_Resume                              0x08004f6b   Thumb Code    22  usbd_core.o(.text)
    USBD_Suspend                             0x08004f81   Thumb Code    28  usbd_core.o(.text)
    USBD_SOF                                 0x08004f9d   Thumb Code    16  usbd_core.o(.text)
    USBD_IsoINIncomplete                     0x08004fd5   Thumb Code    14  usbd_core.o(.text)
    USBD_IsoOUTIncomplete                    0x08004fe3   Thumb Code    14  usbd_core.o(.text)
    .text                                    0x08004ff4   Section        0  usbd_ioreq.o(.text)
    .text                                    0x080050ac   Section        0  usbd_req.o(.text)
    USBD_SetConfig                           0x080050c9   Thumb Code   110  usbd_req.o(.text)
    USBD_GetDescriptor                       0x08005137   Thumb Code   288  usbd_req.o(.text)
    USBD_SetFeature                          0x080054db   Thumb Code   118  usbd_req.o(.text)
    .text                                    0x08005554   Section        0  dadd.o(.text)
    .text                                    0x080056a2   Section        0  dmul.o(.text)
    .text                                    0x08005786   Section        0  ddiv.o(.text)
    .text                                    0x08005864   Section        0  dflti.o(.text)
    .text                                    0x08005886   Section        0  f2d.o(.text)
    .text                                    0x080058ac   Section        0  d2f.o(.text)
    .text                                    0x080058e4   Section        0  llshl.o(.text)
    .text                                    0x08005902   Section        0  llsshr.o(.text)
    .text                                    0x08005926   Section        0  fepilogue.o(.text)
    .text                                    0x08005926   Section        0  iusefp.o(.text)
    .text                                    0x08005994   Section        0  depilogue.o(.text)
    .text                                    0x08005a4e   Section        0  dsqrt.o(.text)
    .text                                    0x08005af0   Section       36  init.o(.text)
    .text                                    0x08005b14   Section        0  llushr.o(.text)
    i.__hardfp_sqrt                          0x08005b34   Section        0  sqrt.o(i.__hardfp_sqrt)
    i.__scatterload_copy                     0x08005bae   Section       14  handlers.o(i.__scatterload_copy)
    i.__scatterload_null                     0x08005bbc   Section        2  handlers.o(i.__scatterload_null)
    i.__scatterload_zeroinit                 0x08005bbe   Section       14  handlers.o(i.__scatterload_zeroinit)
    i.__set_errno                            0x08005bcc   Section        0  errno.o(i.__set_errno)
    i.malloc                                 0x08005bd8   Section        0  malloc.o(i.malloc)
    .constdata                               0x08005c44   Section       28  stm32f4xx_fmc.o(.constdata)
    .data                                    0x20000000   Section       16  stm32f4xx_rcc.o(.data)
    APBAHBPrescTable                         0x20000000   Data          16  stm32f4xx_rcc.o(.data)
    .data                                    0x20000010   Section       16  tm_stm32f4_delay.o(.data)
    .data                                    0x20000020   Section        1  tm_stm32f4_disco.o(.data)
    .data                                    0x20000021   Section        1  stm32f4xx_it.o(.data)
    .data                                    0x20000024   Section       20  system_stm32f4xx.o(.data)
    .data                                    0x20000038   Section        1  tm_stm32f4_sdram.o(.data)
    initialized                              0x20000038   Data           1  tm_stm32f4_sdram.o(.data)
    .data                                    0x2000003c   Section       16  paradaconrolada.o(.data)
    .data                                    0x2000004c   Section       44  usbd_core.o(.data)
    .data                                    0x20000078   Section        4  usbd_core.o(.data)
    .data                                    0x2000007c   Section        4  usbd_core.o(.data)
    .data                                    0x20000080   Section       10  usbd_desc.o(.data)
    .data                                    0x2000008c   Section       16  usbd_req.o(.data)
    cfgidx                                   0x2000008c   Data           1  usbd_req.o(.data)
    .data                                    0x2000009c   Section        4  mvars.o(.data)
    .data                                    0x200000a0   Section        4  mvars.o(.data)
    .data                                    0x200000a4   Section        4  errno.o(.data)
    _errno                                   0x200000a4   Data           4  errno.o(.data)
    .bss                                     0x200000a8   Section       22  tm_stm32f4_gpio.o(.bss)
    GPIO_UsedPins                            0x200000a8   Data          22  tm_stm32f4_gpio.o(.bss)
    .bss                                     0x200000c0   Section      176  main.o(.bss)
    .bss                                     0x20000170   Section     1652  tm_stm32f4_usb_vcp.o(.bss)
    .bss                                     0x200007e4   Section        9  homing.o(.bss)
    HEAP                                     0x200007f0   Section      512  startup_stm32f429_439xx.o(HEAP)
    STACK                                    0x200009f0   Section     1024  startup_stm32f429_439xx.o(STACK)

    Global Symbols

    Symbol Name                              Value     Ov Type        Size  Object(Section)

    BuildAttributes$$THM_ISAv4$E$P$D$K$B$S$7EM$VFPi3$EXTD16$VFPS$VFMA$PE$A:L22UL41UL21$X:L11$S22US41US21$IEEE1$IW$USESV6$~STKCKD$USESV7$~SHL$OTIME$ROPI$IEEEJ$EBA8$MICROLIB$REQ8$PRES8$EABIv2 0x00000000   Number         0  anon$$obj.o ABSOLUTE
    __ARM_use_no_argv                        0x00000000   Number         0  main.o ABSOLUTE
    TM_DELAY_1msHandler                       - Undefined Weak Reference
    __cpp_initialize__aeabi_                  - Undefined Weak Reference
    __cxa_finalize                            - Undefined Weak Reference
    __decompress                              - Undefined Weak Reference
    _clock_init                               - Undefined Weak Reference
    _microlib_exit                            - Undefined Weak Reference
    __Vectors_Size                           0x000001ac   Number         0  startup_stm32f429_439xx.o ABSOLUTE
    __Vectors                                0x08000000   Data           4  startup_stm32f429_439xx.o(RESET)
    __Vectors_End                            0x080001ac   Data           0  startup_stm32f429_439xx.o(RESET)
    __main                                   0x080001ad   Thumb Code     0  entry.o(.ARM.Collect$$$$00000000)
    _main_stk                                0x080001ad   Thumb Code     0  entry2.o(.ARM.Collect$$$$00000001)
    _main_scatterload                        0x080001b1   Thumb Code     0  entry5.o(.ARM.Collect$$$$00000004)
    __main_after_scatterload                 0x080001b5   Thumb Code     0  entry5.o(.ARM.Collect$$$$00000004)
    _main_clock                              0x080001b5   Thumb Code     0  entry7b.o(.ARM.Collect$$$$00000008)
    _main_cpp_init                           0x080001b5   Thumb Code     0  entry8b.o(.ARM.Collect$$$$0000000A)
    _main_init                               0x080001b5   Thumb Code     0  entry9a.o(.ARM.Collect$$$$0000000B)
    __rt_final_cpp                           0x080001bd   Thumb Code     0  entry10a.o(.ARM.Collect$$$$0000000D)
    __rt_final_exit                          0x080001bd   Thumb Code     0  entry11a.o(.ARM.Collect$$$$0000000F)
    Reset_Handler                            0x080001c1   Thumb Code     8  startup_stm32f429_439xx.o(.text)
    ADC_IRQHandler                           0x080001db   Thumb Code     0  startup_stm32f429_439xx.o(.text)
    CAN1_RX0_IRQHandler                      0x080001db   Thumb Code     0  startup_stm32f429_439xx.o(.text)
    CAN1_RX1_IRQHandler                      0x080001db   Thumb Code     0  startup_stm32f429_439xx.o(.text)
    CAN1_SCE_IRQHandler                      0x080001db   Thumb Code     0  startup_stm32f429_439xx.o(.text)
    CAN1_TX_IRQHandler                       0x080001db   Thumb Code     0  startup_stm32f429_439xx.o(.text)
    CAN2_RX0_IRQHandler                      0x080001db   Thumb Code     0  startup_stm32f429_439xx.o(.text)
    CAN2_RX1_IRQHandler                      0x080001db   Thumb Code     0  startup_stm32f429_439xx.o(.text)
    CAN2_SCE_IRQHandler                      0x080001db   Thumb Code     0  startup_stm32f429_439xx.o(.text)
    CAN2_TX_IRQHandler                       0x080001db   Thumb Code     0  startup_stm32f429_439xx.o(.text)
    CRYP_IRQHandler                          0x080001db   Thumb Code     0  startup_stm32f429_439xx.o(.text)
    DCMI_IRQHandler                          0x080001db   Thumb Code     0  startup_stm32f429_439xx.o(.text)
    DMA1_Stream0_IRQHandler                  0x080001db   Thumb Code     0  startup_stm32f429_439xx.o(.text)
    DMA1_Stream1_IRQHandler                  0x080001db   Thumb Code     0  startup_stm32f429_439xx.o(.text)
    DMA1_Stream2_IRQHandler                  0x080001db   Thumb Code     0  startup_stm32f429_439xx.o(.text)
    DMA1_Stream3_IRQHandler                  0x080001db   Thumb Code     0  startup_stm32f429_439xx.o(.text)
    DMA1_Stream4_IRQHandler                  0x080001db   Thumb Code     0  startup_stm32f429_439xx.o(.text)
    DMA1_Stream5_IRQHandler                  0x080001db   Thumb Code     0  startup_stm32f429_439xx.o(.text)
    DMA1_Stream6_IRQHandler                  0x080001db   Thumb Code     0  startup_stm32f429_439xx.o(.text)
    DMA1_Stream7_IRQHandler                  0x080001db   Thumb Code     0  startup_stm32f429_439xx.o(.text)
    DMA2D_IRQHandler                         0x080001db   Thumb Code     0  startup_stm32f429_439xx.o(.text)
    DMA2_Stream0_IRQHandler                  0x080001db   Thumb Code     0  startup_stm32f429_439xx.o(.text)
    DMA2_Stream1_IRQHandler                  0x080001db   Thumb Code     0  startup_stm32f429_439xx.o(.text)
    DMA2_Stream2_IRQHandler                  0x080001db   Thumb Code     0  startup_stm32f429_439xx.o(.text)
    DMA2_Stream3_IRQHandler                  0x080001db   Thumb Code     0  startup_stm32f429_439xx.o(.text)
    DMA2_Stream4_IRQHandler                  0x080001db   Thumb Code     0  startup_stm32f429_439xx.o(.text)
    DMA2_Stream5_IRQHandler                  0x080001db   Thumb Code     0  startup_stm32f429_439xx.o(.text)
    DMA2_Stream6_IRQHandler                  0x080001db   Thumb Code     0  startup_stm32f429_439xx.o(.text)
    DMA2_Stream7_IRQHandler                  0x080001db   Thumb Code     0  startup_stm32f429_439xx.o(.text)
    ETH_IRQHandler                           0x080001db   Thumb Code     0  startup_stm32f429_439xx.o(.text)
    ETH_WKUP_IRQHandler                      0x080001db   Thumb Code     0  startup_stm32f429_439xx.o(.text)
    EXTI15_10_IRQHandler                     0x080001db   Thumb Code     0  startup_stm32f429_439xx.o(.text)
    FLASH_IRQHandler                         0x080001db   Thumb Code     0  startup_stm32f429_439xx.o(.text)
    FMC_IRQHandler                           0x080001db   Thumb Code     0  startup_stm32f429_439xx.o(.text)
    FPU_IRQHandler                           0x080001db   Thumb Code     0  startup_stm32f429_439xx.o(.text)
    HASH_RNG_IRQHandler                      0x080001db   Thumb Code     0  startup_stm32f429_439xx.o(.text)
    I2C1_ER_IRQHandler                       0x080001db   Thumb Code     0  startup_stm32f429_439xx.o(.text)
    I2C1_EV_IRQHandler                       0x080001db   Thumb Code     0  startup_stm32f429_439xx.o(.text)
    I2C2_ER_IRQHandler                       0x080001db   Thumb Code     0  startup_stm32f429_439xx.o(.text)
    I2C2_EV_IRQHandler                       0x080001db   Thumb Code     0  startup_stm32f429_439xx.o(.text)
    I2C3_ER_IRQHandler                       0x080001db   Thumb Code     0  startup_stm32f429_439xx.o(.text)
    I2C3_EV_IRQHandler                       0x080001db   Thumb Code     0  startup_stm32f429_439xx.o(.text)
    LTDC_ER_IRQHandler                       0x080001db   Thumb Code     0  startup_stm32f429_439xx.o(.text)
    LTDC_IRQHandler                          0x080001db   Thumb Code     0  startup_stm32f429_439xx.o(.text)
    OTG_FS_IRQHandler                        0x080001db   Thumb Code     0  startup_stm32f429_439xx.o(.text)
    OTG_FS_WKUP_IRQHandler                   0x080001db   Thumb Code     0  startup_stm32f429_439xx.o(.text)
    PVD_IRQHandler                           0x080001db   Thumb Code     0  startup_stm32f429_439xx.o(.text)
    RCC_IRQHandler                           0x080001db   Thumb Code     0  startup_stm32f429_439xx.o(.text)
    RTC_Alarm_IRQHandler                     0x080001db   Thumb Code     0  startup_stm32f429_439xx.o(.text)
    RTC_WKUP_IRQHandler                      0x080001db   Thumb Code     0  startup_stm32f429_439xx.o(.text)
    SAI1_IRQHandler                          0x080001db   Thumb Code     0  startup_stm32f429_439xx.o(.text)
    SDIO_IRQHandler                          0x080001db   Thumb Code     0  startup_stm32f429_439xx.o(.text)
    SPI1_IRQHandler                          0x080001db   Thumb Code     0  startup_stm32f429_439xx.o(.text)
    SPI2_IRQHandler                          0x080001db   Thumb Code     0  startup_stm32f429_439xx.o(.text)
    SPI3_IRQHandler                          0x080001db   Thumb Code     0  startup_stm32f429_439xx.o(.text)
    SPI4_IRQHandler                          0x080001db   Thumb Code     0  startup_stm32f429_439xx.o(.text)
    SPI5_IRQHandler                          0x080001db   Thumb Code     0  startup_stm32f429_439xx.o(.text)
    SPI6_IRQHandler                          0x080001db   Thumb Code     0  startup_stm32f429_439xx.o(.text)
    TAMP_STAMP_IRQHandler                    0x080001db   Thumb Code     0  startup_stm32f429_439xx.o(.text)
    TIM1_BRK_TIM9_IRQHandler                 0x080001db   Thumb Code     0  startup_stm32f429_439xx.o(.text)
    TIM1_CC_IRQHandler                       0x080001db   Thumb Code     0  startup_stm32f429_439xx.o(.text)
    TIM1_TRG_COM_TIM11_IRQHandler            0x080001db   Thumb Code     0  startup_stm32f429_439xx.o(.text)
    TIM1_UP_TIM10_IRQHandler                 0x080001db   Thumb Code     0  startup_stm32f429_439xx.o(.text)
    TIM3_IRQHandler                          0x080001db   Thumb Code     0  startup_stm32f429_439xx.o(.text)
    TIM4_IRQHandler                          0x080001db   Thumb Code     0  startup_stm32f429_439xx.o(.text)
    TIM5_IRQHandler                          0x080001db   Thumb Code     0  startup_stm32f429_439xx.o(.text)
    TIM6_DAC_IRQHandler                      0x080001db   Thumb Code     0  startup_stm32f429_439xx.o(.text)
    TIM7_IRQHandler                          0x080001db   Thumb Code     0  startup_stm32f429_439xx.o(.text)
    TIM8_BRK_TIM12_IRQHandler                0x080001db   Thumb Code     0  startup_stm32f429_439xx.o(.text)
    TIM8_CC_IRQHandler                       0x080001db   Thumb Code     0  startup_stm32f429_439xx.o(.text)
    TIM8_TRG_COM_TIM14_IRQHandler            0x080001db   Thumb Code     0  startup_stm32f429_439xx.o(.text)
    TIM8_UP_TIM13_IRQHandler                 0x080001db   Thumb Code     0  startup_stm32f429_439xx.o(.text)
    UART4_IRQHandler                         0x080001db   Thumb Code     0  startup_stm32f429_439xx.o(.text)
    UART5_IRQHandler                         0x080001db   Thumb Code     0  startup_stm32f429_439xx.o(.text)
    UART7_IRQHandler                         0x080001db   Thumb Code     0  startup_stm32f429_439xx.o(.text)
    UART8_IRQHandler                         0x080001db   Thumb Code     0  startup_stm32f429_439xx.o(.text)
    USART1_IRQHandler                        0x080001db   Thumb Code     0  startup_stm32f429_439xx.o(.text)
    USART2_IRQHandler                        0x080001db   Thumb Code     0  startup_stm32f429_439xx.o(.text)
    USART3_IRQHandler                        0x080001db   Thumb Code     0  startup_stm32f429_439xx.o(.text)
    USART6_IRQHandler                        0x080001db   Thumb Code     0  startup_stm32f429_439xx.o(.text)
    WWDG_IRQHandler                          0x080001db   Thumb Code     0  startup_stm32f429_439xx.o(.text)
    NVIC_PriorityGroupConfig                 0x080001e5   Thumb Code    10  misc.o(.text)
    NVIC_Init                                0x080001ef   Thumb Code    96  misc.o(.text)
    NVIC_SetVectorTable                      0x0800024f   Thumb Code    14  misc.o(.text)
    NVIC_SystemLPConfig                      0x0800025d   Thumb Code    20  misc.o(.text)
    SysTick_CLKSourceConfig                  0x08000271   Thumb Code    24  misc.o(.text)
    RCC_DeInit                               0x08000295   Thumb Code    68  stm32f4xx_rcc.o(.text)
    RCC_HSEConfig                            0x080002d9   Thumb Code    12  stm32f4xx_rcc.o(.text)
    RCC_GetFlagStatus                        0x080002e5   Thumb Code    46  stm32f4xx_rcc.o(.text)
    RCC_WaitForHSEStartUp                    0x08000313   Thumb Code    44  stm32f4xx_rcc.o(.text)
    RCC_AdjustHSICalibrationValue            0x0800033f   Thumb Code    16  stm32f4xx_rcc.o(.text)
    RCC_HSICmd                               0x0800034f   Thumb Code     6  stm32f4xx_rcc.o(.text)
    RCC_LSEConfig                            0x08000355   Thumb Code    24  stm32f4xx_rcc.o(.text)
    RCC_LSICmd                               0x0800036d   Thumb Code     6  stm32f4xx_rcc.o(.text)
    RCC_PLLConfig                            0x08000373   Thumb Code    32  stm32f4xx_rcc.o(.text)
    RCC_PLLCmd                               0x08000393   Thumb Code     6  stm32f4xx_rcc.o(.text)
    RCC_PLLI2SConfig                         0x08000399   Thumb Code    18  stm32f4xx_rcc.o(.text)
    RCC_PLLI2SCmd                            0x080003ab   Thumb Code     6  stm32f4xx_rcc.o(.text)
    RCC_PLLSAIConfig                         0x080003b1   Thumb Code    18  stm32f4xx_rcc.o(.text)
    RCC_PLLSAICmd                            0x080003c3   Thumb Code     6  stm32f4xx_rcc.o(.text)
    RCC_ClockSecuritySystemCmd               0x080003c9   Thumb Code     6  stm32f4xx_rcc.o(.text)
    RCC_MCO1Config                           0x080003cf   Thumb Code    18  stm32f4xx_rcc.o(.text)
    RCC_MCO2Config                           0x080003e1   Thumb Code    18  stm32f4xx_rcc.o(.text)
    RCC_SYSCLKConfig                         0x080003f3   Thumb Code    16  stm32f4xx_rcc.o(.text)
    RCC_GetSYSCLKSource                      0x08000403   Thumb Code    12  stm32f4xx_rcc.o(.text)
    RCC_HCLKConfig                           0x0800040f   Thumb Code    16  stm32f4xx_rcc.o(.text)
    RCC_PCLK1Config                          0x0800041f   Thumb Code    16  stm32f4xx_rcc.o(.text)
    RCC_PCLK2Config                          0x0800042f   Thumb Code    18  stm32f4xx_rcc.o(.text)
    RCC_GetClocksFreq                        0x08000441   Thumb Code   134  stm32f4xx_rcc.o(.text)
    RCC_RTCCLKConfig                         0x080004c7   Thumb Code    42  stm32f4xx_rcc.o(.text)
    RCC_RTCCLKCmd                            0x080004f1   Thumb Code     8  stm32f4xx_rcc.o(.text)
    RCC_BackupResetCmd                       0x080004f9   Thumb Code     8  stm32f4xx_rcc.o(.text)
    RCC_I2SCLKConfig                         0x08000501   Thumb Code     8  stm32f4xx_rcc.o(.text)
    RCC_SAIBlockACLKConfig                   0x08000509   Thumb Code    16  stm32f4xx_rcc.o(.text)
    RCC_SAIBlockBCLKConfig                   0x08000519   Thumb Code    16  stm32f4xx_rcc.o(.text)
    RCC_SAIPLLI2SClkDivConfig                0x08000529   Thumb Code    18  stm32f4xx_rcc.o(.text)
    RCC_SAIPLLSAIClkDivConfig                0x0800053b   Thumb Code    24  stm32f4xx_rcc.o(.text)
    RCC_LTDCCLKDivConfig                     0x08000553   Thumb Code    16  stm32f4xx_rcc.o(.text)
    RCC_TIMCLKPresConfig                     0x08000563   Thumb Code     8  stm32f4xx_rcc.o(.text)
    RCC_AHB1PeriphClockCmd                   0x0800056b   Thumb Code    20  stm32f4xx_rcc.o(.text)
    RCC_AHB2PeriphClockCmd                   0x0800057f   Thumb Code    20  stm32f4xx_rcc.o(.text)
    RCC_AHB3PeriphClockCmd                   0x08000593   Thumb Code    20  stm32f4xx_rcc.o(.text)
    RCC_APB1PeriphClockCmd                   0x080005a7   Thumb Code    20  stm32f4xx_rcc.o(.text)
    RCC_APB2PeriphClockCmd                   0x080005bb   Thumb Code    20  stm32f4xx_rcc.o(.text)
    RCC_AHB1PeriphResetCmd                   0x080005cf   Thumb Code    20  stm32f4xx_rcc.o(.text)
    RCC_AHB2PeriphResetCmd                   0x080005e3   Thumb Code    20  stm32f4xx_rcc.o(.text)
    RCC_AHB3PeriphResetCmd                   0x080005f7   Thumb Code    20  stm32f4xx_rcc.o(.text)
    RCC_APB1PeriphResetCmd                   0x0800060b   Thumb Code    20  stm32f4xx_rcc.o(.text)
    RCC_APB2PeriphResetCmd                   0x0800061f   Thumb Code    20  stm32f4xx_rcc.o(.text)
    RCC_AHB1PeriphClockLPModeCmd             0x08000633   Thumb Code    20  stm32f4xx_rcc.o(.text)
    RCC_AHB2PeriphClockLPModeCmd             0x08000647   Thumb Code    20  stm32f4xx_rcc.o(.text)
    RCC_AHB3PeriphClockLPModeCmd             0x0800065b   Thumb Code    20  stm32f4xx_rcc.o(.text)
    RCC_APB1PeriphClockLPModeCmd             0x0800066f   Thumb Code    64  stm32f4xx_rcc.o(.text)
    RCC_APB2PeriphClockLPModeCmd             0x080006af   Thumb Code    18  stm32f4xx_rcc.o(.text)
    RCC_LSEModeConfig                        0x080006c1   Thumb Code    24  stm32f4xx_rcc.o(.text)
    RCC_ITConfig                             0x080006d9   Thumb Code    20  stm32f4xx_rcc.o(.text)
    RCC_ClearFlag                            0x080006ed   Thumb Code    14  stm32f4xx_rcc.o(.text)
    RCC_GetITStatus                          0x080006fb   Thumb Code    18  stm32f4xx_rcc.o(.text)
    RCC_ClearITPendingBit                    0x0800070d   Thumb Code     8  stm32f4xx_rcc.o(.text)
    GPIO_DeInit                              0x08000719   Thumb Code   216  stm32f4xx_gpio.o(.text)
    GPIO_Init                                0x080007f1   Thumb Code   120  stm32f4xx_gpio.o(.text)
    GPIO_StructInit                          0x08000869   Thumb Code    18  stm32f4xx_gpio.o(.text)
    GPIO_PinLockConfig                       0x0800087b   Thumb Code    24  stm32f4xx_gpio.o(.text)
    GPIO_ReadInputDataBit                    0x08000893   Thumb Code    14  stm32f4xx_gpio.o(.text)
    GPIO_ReadInputData                       0x080008a1   Thumb Code     6  stm32f4xx_gpio.o(.text)
    GPIO_ReadOutputDataBit                   0x080008a7   Thumb Code    14  stm32f4xx_gpio.o(.text)
    GPIO_ReadOutputData                      0x080008b5   Thumb Code     6  stm32f4xx_gpio.o(.text)
    GPIO_SetBits                             0x080008bb   Thumb Code     4  stm32f4xx_gpio.o(.text)
    GPIO_ResetBits                           0x080008bf   Thumb Code     4  stm32f4xx_gpio.o(.text)
    GPIO_WriteBit                            0x080008c3   Thumb Code    10  stm32f4xx_gpio.o(.text)
    GPIO_Write                               0x080008cd   Thumb Code     4  stm32f4xx_gpio.o(.text)
    GPIO_ToggleBits                          0x080008d1   Thumb Code     8  stm32f4xx_gpio.o(.text)
    GPIO_PinAFConfig                         0x080008d9   Thumb Code    32  stm32f4xx_gpio.o(.text)
    EXTI_DeInit                              0x08000925   Thumb Code    28  stm32f4xx_exti.o(.text)
    EXTI_Init                                0x08000941   Thumb Code   108  stm32f4xx_exti.o(.text)
    EXTI_StructInit                          0x080009ad   Thumb Code    14  stm32f4xx_exti.o(.text)
    EXTI_GenerateSWInterrupt                 0x080009bb   Thumb Code    12  stm32f4xx_exti.o(.text)
    EXTI_GetFlagStatus                       0x080009c7   Thumb Code    18  stm32f4xx_exti.o(.text)
    EXTI_ClearFlag                           0x080009d9   Thumb Code     8  stm32f4xx_exti.o(.text)
    EXTI_GetITStatus                         0x080009e1   Thumb Code    18  stm32f4xx_exti.o(.text)
    EXTI_ClearITPendingBit                   0x080009f3   Thumb Code     8  stm32f4xx_exti.o(.text)
    TIM_DeInit                               0x08000a05   Thumb Code   284  stm32f4xx_tim.o(.text)
    TIM_TimeBaseInit                         0x08000b21   Thumb Code    96  stm32f4xx_tim.o(.text)
    TIM_TimeBaseStructInit                   0x08000b81   Thumb Code    18  stm32f4xx_tim.o(.text)
    TIM_PrescalerConfig                      0x08000b93   Thumb Code     6  stm32f4xx_tim.o(.text)
    TIM_CounterModeConfig                    0x08000b99   Thumb Code    12  stm32f4xx_tim.o(.text)
    TIM_SetCounter                           0x08000ba5   Thumb Code     4  stm32f4xx_tim.o(.text)
    TIM_SetAutoreload                        0x08000ba9   Thumb Code     4  stm32f4xx_tim.o(.text)
    TIM_GetCounter                           0x08000bad   Thumb Code     4  stm32f4xx_tim.o(.text)
    TIM_GetPrescaler                         0x08000bb1   Thumb Code     4  stm32f4xx_tim.o(.text)
    TIM_UpdateDisableConfig                  0x08000bb5   Thumb Code    20  stm32f4xx_tim.o(.text)
    TIM_UpdateRequestConfig                  0x08000bc9   Thumb Code    20  stm32f4xx_tim.o(.text)
    TIM_ARRPreloadConfig                     0x08000bdd   Thumb Code    20  stm32f4xx_tim.o(.text)
    TIM_SelectOnePulseMode                   0x08000bf1   Thumb Code    16  stm32f4xx_tim.o(.text)
    TIM_SetClockDivision                     0x08000c01   Thumb Code    16  stm32f4xx_tim.o(.text)
    TIM_Cmd                                  0x08000c11   Thumb Code    20  stm32f4xx_tim.o(.text)
    TIM_OC1Init                              0x08000c25   Thumb Code    88  stm32f4xx_tim.o(.text)
    TIM_OC2Init                              0x08000c7d   Thumb Code   120  stm32f4xx_tim.o(.text)
    TIM_OC3Init                              0x08000cf5   Thumb Code   116  stm32f4xx_tim.o(.text)
    TIM_OC4Init                              0x08000d69   Thumb Code    88  stm32f4xx_tim.o(.text)
    TIM_OCStructInit                         0x08000dc1   Thumb Code    20  stm32f4xx_tim.o(.text)
    TIM_SelectOCxM                           0x08000dd5   Thumb Code   130  stm32f4xx_tim.o(.text)
    TIM_SetCompare1                          0x08000e57   Thumb Code     4  stm32f4xx_tim.o(.text)
    TIM_SetCompare2                          0x08000e5b   Thumb Code     4  stm32f4xx_tim.o(.text)
    TIM_SetCompare3                          0x08000e5f   Thumb Code     4  stm32f4xx_tim.o(.text)
    TIM_SetCompare4                          0x08000e63   Thumb Code     4  stm32f4xx_tim.o(.text)
    TIM_ForcedOC1Config                      0x08000e67   Thumb Code    12  stm32f4xx_tim.o(.text)
    TIM_ForcedOC2Config                      0x08000e73   Thumb Code    20  stm32f4xx_tim.o(.text)
    TIM_ForcedOC3Config                      0x08000e87   Thumb Code    12  stm32f4xx_tim.o(.text)
    TIM_ForcedOC4Config                      0x08000e93   Thumb Code    20  stm32f4xx_tim.o(.text)
    TIM_OC1PreloadConfig                     0x08000ea7   Thumb Code    12  stm32f4xx_tim.o(.text)
    TIM_OC2PreloadConfig                     0x08000eb3   Thumb Code    20  stm32f4xx_tim.o(.text)
    TIM_OC3PreloadConfig                     0x08000ec7   Thumb Code    12  stm32f4xx_tim.o(.text)
    TIM_OC4PreloadConfig                     0x08000ed3   Thumb Code    20  stm32f4xx_tim.o(.text)
    TIM_OC1FastConfig                        0x08000ee7   Thumb Code    12  stm32f4xx_tim.o(.text)
    TIM_OC2FastConfig                        0x08000ef3   Thumb Code    20  stm32f4xx_tim.o(.text)
    TIM_OC3FastConfig                        0x08000f07   Thumb Code    12  stm32f4xx_tim.o(.text)
    TIM_OC4FastConfig                        0x08000f13   Thumb Code    20  stm32f4xx_tim.o(.text)
    TIM_ClearOC1Ref                          0x08000f27   Thumb Code    12  stm32f4xx_tim.o(.text)
    TIM_ClearOC2Ref                          0x08000f33   Thumb Code    20  stm32f4xx_tim.o(.text)
    TIM_ClearOC3Ref                          0x08000f47   Thumb Code    12  stm32f4xx_tim.o(.text)
    TIM_ClearOC4Ref                          0x08000f53   Thumb Code    20  stm32f4xx_tim.o(.text)
    TIM_OC1PolarityConfig                    0x08000f67   Thumb Code    12  stm32f4xx_tim.o(.text)
    TIM_OC1NPolarityConfig                   0x08000f73   Thumb Code    12  stm32f4xx_tim.o(.text)
    TIM_OC2PolarityConfig                    0x08000f7f   Thumb Code    20  stm32f4xx_tim.o(.text)
    TIM_OC2NPolarityConfig                   0x08000f93   Thumb Code    20  stm32f4xx_tim.o(.text)
    TIM_OC3PolarityConfig                    0x08000fa7   Thumb Code    20  stm32f4xx_tim.o(.text)
    TIM_OC3NPolarityConfig                   0x08000fbb   Thumb Code    20  stm32f4xx_tim.o(.text)
    TIM_OC4PolarityConfig                    0x08000fcf   Thumb Code    20  stm32f4xx_tim.o(.text)
    TIM_CCxCmd                               0x08000fe3   Thumb Code    22  stm32f4xx_tim.o(.text)
    TIM_CCxNCmd                              0x08000ff9   Thumb Code    22  stm32f4xx_tim.o(.text)
    TIM_SetIC4Prescaler                      0x0800100f   Thumb Code    24  stm32f4xx_tim.o(.text)
    TIM_SetIC3Prescaler                      0x08001027   Thumb Code    16  stm32f4xx_tim.o(.text)
    TIM_SetIC2Prescaler                      0x08001037   Thumb Code    24  stm32f4xx_tim.o(.text)
    TIM_SetIC1Prescaler                      0x08001085   Thumb Code    16  stm32f4xx_tim.o(.text)
    TIM_ICInit                               0x08001095   Thumb Code   164  stm32f4xx_tim.o(.text)
    TIM_ICStructInit                         0x08001139   Thumb Code    16  stm32f4xx_tim.o(.text)
    TIM_PWMIConfig                           0x08001149   Thumb Code   104  stm32f4xx_tim.o(.text)
    TIM_GetCapture1                          0x080011b1   Thumb Code     4  stm32f4xx_tim.o(.text)
    TIM_GetCapture2                          0x080011b5   Thumb Code     4  stm32f4xx_tim.o(.text)
    TIM_GetCapture3                          0x080011b9   Thumb Code     4  stm32f4xx_tim.o(.text)
    TIM_GetCapture4                          0x080011bd   Thumb Code     4  stm32f4xx_tim.o(.text)
    TIM_BDTRConfig                           0x080011c1   Thumb Code    34  stm32f4xx_tim.o(.text)
    TIM_BDTRStructInit                       0x080011e3   Thumb Code    18  stm32f4xx_tim.o(.text)
    TIM_CtrlPWMOutputs                       0x080011f5   Thumb Code    22  stm32f4xx_tim.o(.text)
    TIM_SelectCOM                            0x0800120b   Thumb Code    20  stm32f4xx_tim.o(.text)
    TIM_CCPreloadControl                     0x0800121f   Thumb Code    20  stm32f4xx_tim.o(.text)
    TIM_ITConfig                             0x08001233   Thumb Code    16  stm32f4xx_tim.o(.text)
    TIM_GenerateEvent                        0x08001243   Thumb Code     4  stm32f4xx_tim.o(.text)
    TIM_GetFlagStatus                        0x08001247   Thumb Code    14  stm32f4xx_tim.o(.text)
    TIM_ClearFlag                            0x08001255   Thumb Code     6  stm32f4xx_tim.o(.text)
    TIM_GetITStatus                          0x0800125b   Thumb Code    24  stm32f4xx_tim.o(.text)
    TIM_ClearITPendingBit                    0x08001273   Thumb Code     6  stm32f4xx_tim.o(.text)
    TIM_DMAConfig                            0x08001279   Thumb Code     8  stm32f4xx_tim.o(.text)
    TIM_DMACmd                               0x08001281   Thumb Code    16  stm32f4xx_tim.o(.text)
    TIM_SelectCCDMA                          0x08001291   Thumb Code    20  stm32f4xx_tim.o(.text)
    TIM_InternalClockConfig                  0x080012a5   Thumb Code    10  stm32f4xx_tim.o(.text)
    TIM_SelectInputTrigger                   0x080012af   Thumb Code    12  stm32f4xx_tim.o(.text)
    TIM_ITRxExternalClockConfig              0x080012bb   Thumb Code    18  stm32f4xx_tim.o(.text)
    TIM_TIxExternalClockConfig               0x080012cd   Thumb Code    46  stm32f4xx_tim.o(.text)
    TIM_ETRConfig                            0x080012fb   Thumb Code    24  stm32f4xx_tim.o(.text)
    TIM_ETRClockMode1Config                  0x08001313   Thumb Code    18  stm32f4xx_tim.o(.text)
    TIM_ETRClockMode2Config                  0x08001325   Thumb Code    18  stm32f4xx_tim.o(.text)
    TIM_SelectOutputTrigger                  0x08001337   Thumb Code    16  stm32f4xx_tim.o(.text)
    TIM_SelectSlaveMode                      0x08001347   Thumb Code    16  stm32f4xx_tim.o(.text)
    TIM_SelectMasterSlaveMode                0x08001357   Thumb Code    16  stm32f4xx_tim.o(.text)
    TIM_EncoderInterfaceConfig               0x08001367   Thumb Code    50  stm32f4xx_tim.o(.text)
    TIM_SelectHallSensor                     0x08001399   Thumb Code    20  stm32f4xx_tim.o(.text)
    TIM_RemapConfig                          0x080013ad   Thumb Code     6  stm32f4xx_tim.o(.text)
    DAC_DeInit                               0x080013e1   Thumb Code    24  stm32f4xx_dac.o(.text)
    DAC_Init                                 0x080013f9   Thumb Code    36  stm32f4xx_dac.o(.text)
    DAC_StructInit                           0x0800141d   Thumb Code    12  stm32f4xx_dac.o(.text)
    DAC_Cmd                                  0x08001429   Thumb Code    20  stm32f4xx_dac.o(.text)
    DAC_SoftwareTriggerCmd                   0x0800143d   Thumb Code    26  stm32f4xx_dac.o(.text)
    DAC_DualSoftwareTriggerCmd               0x08001457   Thumb Code    24  stm32f4xx_dac.o(.text)
    DAC_WaveGenerationCmd                    0x0800146f   Thumb Code    18  stm32f4xx_dac.o(.text)
    DAC_SetChannel1Data                      0x08001481   Thumb Code    14  stm32f4xx_dac.o(.text)
    DAC_SetChannel2Data                      0x0800148f   Thumb Code    14  stm32f4xx_dac.o(.text)
    DAC_SetDualChannelData                   0x0800149d   Thumb Code    22  stm32f4xx_dac.o(.text)
    DAC_GetDataOutputValue                   0x080014b3   Thumb Code    18  stm32f4xx_dac.o(.text)
    DAC_DMACmd                               0x080014c5   Thumb Code    20  stm32f4xx_dac.o(.text)
    DAC_ITConfig                             0x080014d9   Thumb Code    18  stm32f4xx_dac.o(.text)
    DAC_GetFlagStatus                        0x080014eb   Thumb Code    20  stm32f4xx_dac.o(.text)
    DAC_ClearFlag                            0x080014ff   Thumb Code    10  stm32f4xx_dac.o(.text)
    DAC_GetITStatus                          0x08001509   Thumb Code    30  stm32f4xx_dac.o(.text)
    DAC_ClearITPendingBit                    0x08001527   Thumb Code    10  stm32f4xx_dac.o(.text)
    SYSCFG_DeInit                            0x08001535   Thumb Code    24  stm32f4xx_syscfg.o(.text)
    SYSCFG_MemoryRemapConfig                 0x0800154d   Thumb Code     6  stm32f4xx_syscfg.o(.text)
    SYSCFG_MemorySwappingBank                0x08001553   Thumb Code     6  stm32f4xx_syscfg.o(.text)
    SYSCFG_EXTILineConfig                    0x08001559   Thumb Code    42  stm32f4xx_syscfg.o(.text)
    SYSCFG_ETH_MediaInterfaceConfig          0x08001583   Thumb Code     8  stm32f4xx_syscfg.o(.text)
    SYSCFG_CompensationCellCmd               0x0800158b   Thumb Code     6  stm32f4xx_syscfg.o(.text)
    SYSCFG_GetCompensationCellStatus         0x08001591   Thumb Code    16  stm32f4xx_syscfg.o(.text)
    FMC_NORSRAMDeInit                        0x080015b1   Thumb Code    38  stm32f4xx_fmc.o(.text)
    FMC_NORSRAMInit                          0x080015d7   Thumb Code   264  stm32f4xx_fmc.o(.text)
    FMC_NORSRAMStructInit                    0x080016df   Thumb Code    46  stm32f4xx_fmc.o(.text)
    FMC_NORSRAMCmd                           0x0800170d   Thumb Code    26  stm32f4xx_fmc.o(.text)
    FMC_NANDDeInit                           0x08001727   Thumb Code    40  stm32f4xx_fmc.o(.text)
    FMC_NANDInit                             0x0800174f   Thumb Code   158  stm32f4xx_fmc.o(.text)
    FMC_NANDStructInit                       0x080017ed   Thumb Code    54  stm32f4xx_fmc.o(.text)
    FMC_NANDCmd                              0x08001823   Thumb Code    54  stm32f4xx_fmc.o(.text)
    FMC_NANDECCCmd                           0x08001859   Thumb Code    54  stm32f4xx_fmc.o(.text)
    FMC_GetECC                               0x0800188f   Thumb Code    18  stm32f4xx_fmc.o(.text)
    FMC_PCCARDDeInit                         0x080018a1   Thumb Code    26  stm32f4xx_fmc.o(.text)
    FMC_PCCARDInit                           0x080018bb   Thumb Code   116  stm32f4xx_fmc.o(.text)
    FMC_PCCARDStructInit                     0x0800192f   Thumb Code    60  stm32f4xx_fmc.o(.text)
    FMC_PCCARDCmd                            0x0800196b   Thumb Code    28  stm32f4xx_fmc.o(.text)
    FMC_SDRAMDeInit                          0x08001987   Thumb Code    42  stm32f4xx_fmc.o(.text)
    FMC_SDRAMInit                            0x080019b1   Thumb Code   308  stm32f4xx_fmc.o(.text)
    FMC_SDRAMStructInit                      0x08001ae5   Thumb Code    60  stm32f4xx_fmc.o(.text)
    FMC_SDRAMCmdConfig                       0x08001b21   Thumb Code    34  stm32f4xx_fmc.o(.text)
    FMC_GetModeStatus                        0x08001b43   Thumb Code    26  stm32f4xx_fmc.o(.text)
    FMC_SetRefreshCount                      0x08001b5d   Thumb Code    18  stm32f4xx_fmc.o(.text)
    FMC_SetAutoRefresh_Number                0x08001b6f   Thumb Code    18  stm32f4xx_fmc.o(.text)
    FMC_SDRAMWriteProtectionConfig           0x08001b81   Thumb Code    32  stm32f4xx_fmc.o(.text)
    FMC_ITConfig                             0x08001ba1   Thumb Code   102  stm32f4xx_fmc.o(.text)
    FMC_GetFlagStatus                        0x08001c07   Thumb Code    54  stm32f4xx_fmc.o(.text)
    FMC_ClearFlag                            0x08001c3d   Thumb Code    56  stm32f4xx_fmc.o(.text)
    FMC_GetITStatus                          0x08001c75   Thumb Code    80  stm32f4xx_fmc.o(.text)
    FMC_ClearITPendingBit                    0x08001cc5   Thumb Code    62  stm32f4xx_fmc.o(.text)
    TimingDelay_Decrement                    0x08001d09   Thumb Code    26  tm_stm32f4_delay.o(.text)
    TM_DELAY_Init                            0x08001d23   Thumb Code    82  tm_stm32f4_delay.o(.text)
    TM_DELAY_EnableDelayTimer                0x08001d75   Thumb Code    22  tm_stm32f4_delay.o(.text)
    TM_DELAY_DisableDelayTimer               0x08001d8b   Thumb Code    14  tm_stm32f4_delay.o(.text)
    TM_DISCO_LedInit                         0x08001da9   Thumb Code    48  tm_stm32f4_disco.o(.text)
    TM_DISCO_ButtonInit                      0x08001dd9   Thumb Code    44  tm_stm32f4_disco.o(.text)
    TM_DISCO_ButtonOnPressed                 0x08001e05   Thumb Code    26  tm_stm32f4_disco.o(.text)
    TM_DISCO_ButtonOnReleased                0x08001e1f   Thumb Code    26  tm_stm32f4_disco.o(.text)
    TM_GPIO_GetPortSource                    0x08001e45   Thumb Code    10  tm_stm32f4_gpio.o(.text)
    TM_GPIO_INT_Init                         0x08001e4f   Thumb Code   130  tm_stm32f4_gpio.o(.text)
    TM_GPIO_INT_EnableClock                  0x08001ed1   Thumb Code    20  tm_stm32f4_gpio.o(.text)
    TM_GPIO_Init                             0x08001ee5   Thumb Code    34  tm_stm32f4_gpio.o(.text)
    TM_GPIO_InitAlternate                    0x08001f07   Thumb Code    92  tm_stm32f4_gpio.o(.text)
    TM_GPIO_DeInit                           0x08001f63   Thumb Code    66  tm_stm32f4_gpio.o(.text)
    TM_GPIO_SetPinAsInput                    0x08001fa5   Thumb Code    38  tm_stm32f4_gpio.o(.text)
    TM_GPIO_SetPinAsOutput                   0x08001fcb   Thumb Code    46  tm_stm32f4_gpio.o(.text)
    TM_GPIO_SetPinAsAnalog                   0x08001ff9   Thumb Code    38  tm_stm32f4_gpio.o(.text)
    TM_GPIO_SetPinAsAlternate                0x0800201f   Thumb Code    48  tm_stm32f4_gpio.o(.text)
    TM_GPIO_SetPullResistor                  0x0800204f   Thumb Code    46  tm_stm32f4_gpio.o(.text)
    TM_GPIO_Lock                             0x0800207d   Thumb Code    16  tm_stm32f4_gpio.o(.text)
    TM_GPIO_GetPinSource                     0x0800208d   Thumb Code    18  tm_stm32f4_gpio.o(.text)
    TM_GPIO_INT_DisableClock                 0x0800209f   Thumb Code    20  tm_stm32f4_gpio.o(.text)
    TM_GPIO_GetUsedPins                      0x080020b3   Thumb Code    14  tm_stm32f4_gpio.o(.text)
    TM_GPIO_GetFreePins                      0x080020c1   Thumb Code    18  tm_stm32f4_gpio.o(.text)
    main                                     0x080020e1   Thumb Code   244  main.o(.text)
    NMI_Handler                              0x08002209   Thumb Code     2  stm32f4xx_it.o(.text)
    HardFault_Handler                        0x0800220b   Thumb Code     2  stm32f4xx_it.o(.text)
    MemManage_Handler                        0x0800220d   Thumb Code     2  stm32f4xx_it.o(.text)
    BusFault_Handler                         0x0800220f   Thumb Code     2  stm32f4xx_it.o(.text)
    UsageFault_Handler                       0x08002211   Thumb Code     2  stm32f4xx_it.o(.text)
    SVC_Handler                              0x08002213   Thumb Code     2  stm32f4xx_it.o(.text)
    DebugMon_Handler                         0x08002215   Thumb Code     2  stm32f4xx_it.o(.text)
    PendSV_Handler                           0x08002217   Thumb Code     2  stm32f4xx_it.o(.text)
    SysTick_Handler                          0x0800221b   Thumb Code     8  stm32f4xx_it.o(.text)
    TIM2_IRQHandler                          0x08002223   Thumb Code    36  stm32f4xx_it.o(.text)
    EXTI0_IRQHandler                         0x08002247   Thumb Code    54  stm32f4xx_it.o(.text)
    EXTI1_IRQHandler                         0x0800227d   Thumb Code    54  stm32f4xx_it.o(.text)
    EXTI2_IRQHandler                         0x080022b3   Thumb Code    38  stm32f4xx_it.o(.text)
    EXTI3_IRQHandler                         0x080022d9   Thumb Code    38  stm32f4xx_it.o(.text)
    EXTI4_IRQHandler                         0x080022ff   Thumb Code    62  stm32f4xx_it.o(.text)
    EXTI9_5_IRQHandler                       0x0800233d   Thumb Code    62  stm32f4xx_it.o(.text)
    SystemInit                               0x08002457   Thumb Code    74  system_stm32f4xx.o(.text)
    SystemCoreClockUpdate                    0x080024a1   Thumb Code   108  system_stm32f4xx.o(.text)
    TM_SDRAM_InitCustomPinsCallback          0x08002531   Thumb Code     4  tm_stm32f4_sdram.o(.text)
    TM_SDRAM_Init                            0x08002535   Thumb Code   368  tm_stm32f4_sdram.o(.text)
    Control_TimerInit                        0x08002741   Thumb Code   124  config.o(.text)
    encoder1_config                          0x080027bd   Thumb Code   138  config.o(.text)
    encoder2_config                          0x08002847   Thumb Code   136  config.o(.text)
    encoder3_config                          0x080028cf   Thumb Code   134  config.o(.text)
    encoder4_config                          0x08002955   Thumb Code   134  config.o(.text)
    dac_init                                 0x080029db   Thumb Code    98  config.o(.text)
    PWM                                      0x08002a3d   Thumb Code   336  config.o(.text)
    Configure_GPIOB_EXTI                     0x08002b8d   Thumb Code   208  config.o(.text)
    Configure_GPIOF_EXTI                     0x08002c5d   Thumb Code   148  config.o(.text)
    check_sign                               0x08002cf9   Thumb Code    20  trapez.o(.text)
    trapez4                                  0x08002d0d   Thumb Code  2042  trapez.o(.text)
    trapez                                   0x08003507   Thumb Code   854  trapez.o(.text)
    vel_reference                            0x08003869   Thumb Code    50  functions.o(.text)
    speed_estimation                         0x0800389b   Thumb Code    10  functions.o(.text)
    PPR_to_Rad                               0x080038a5   Thumb Code   114  functions.o(.text)
    escalado                                 0x08003917   Thumb Code    38  functions.o(.text)
    PI_action                                0x08003965   Thumb Code    44  controller.o(.text)
    PD_action                                0x08003991   Thumb Code    40  controller.o(.text)
    paradacontrolada                         0x080039c1   Thumb Code   266  paradaconrolada.o(.text)
    USB_OTG_BSP_Init                         0x08003ae9   Thumb Code   170  usb_bsp.o(.text)
    USB_OTG_BSP_EnableInterrupt              0x08003b93   Thumb Code   104  usb_bsp.o(.text)
    USB_OTG_BSP_uDelay                       0x08003bfb   Thumb Code    22  usb_bsp.o(.text)
    USB_OTG_BSP_mDelay                       0x08003c11   Thumb Code     8  usb_bsp.o(.text)
    OTG_HS_WKUP_IRQHandler                   0x08003c19   Thumb Code     8  usb_bsp.o(.text)
    OTG_HS_IRQHandler                        0x08003c21   Thumb Code     6  usb_bsp.o(.text)
    OTG_HS_EP1_IN_IRQHandler                 0x08003c27   Thumb Code     6  usb_bsp.o(.text)
    OTG_HS_EP1_OUT_IRQHandler                0x08003c2d   Thumb Code     6  usb_bsp.o(.text)
    USB_OTG_WritePacket                      0x08003c91   Thumb Code    40  usb_core.o(.text)
    USB_OTG_ReadPacket                       0x08003cb9   Thumb Code    32  usb_core.o(.text)
    USB_OTG_SelectCore                       0x08003cd9   Thumb Code   192  usb_core.o(.text)
    USB_OTG_CoreInit                         0x08003d99   Thumb Code   128  usb_core.o(.text)
    USB_OTG_EnableGlobalInt                  0x08003e19   Thumb Code    16  usb_core.o(.text)
    USB_OTG_DisableGlobalInt                 0x08003e29   Thumb Code    16  usb_core.o(.text)
    USB_OTG_FlushTxFifo                      0x08003e39   Thumb Code    62  usb_core.o(.text)
    USB_OTG_FlushRxFifo                      0x08003e77   Thumb Code    54  usb_core.o(.text)
    USB_OTG_SetCurrentMode                   0x08003ead   Thumb Code    42  usb_core.o(.text)
    USB_OTG_GetMode                          0x08003ed7   Thumb Code    10  usb_core.o(.text)
    USB_OTG_IsDeviceMode                     0x08003ee1   Thumb Code    18  usb_core.o(.text)
    USB_OTG_IsHostMode                       0x08003ef3   Thumb Code    14  usb_core.o(.text)
    USB_OTG_ReadCoreItr                      0x08003f01   Thumb Code    10  usb_core.o(.text)
    USB_OTG_ReadOtgItr                       0x08003f0b   Thumb Code     6  usb_core.o(.text)
    USB_OTG_InitDevSpeed                     0x08003f11   Thumb Code    12  usb_core.o(.text)
    USB_OTG_EnableDevInt                     0x08003f1d   Thumb Code    66  usb_core.o(.text)
    USB_OTG_CoreInitDev                      0x08003f5f   Thumb Code   364  usb_core.o(.text)
    USB_OTG_GetDeviceSpeed                   0x080040cb   Thumb Code    38  usb_core.o(.text)
    USB_OTG_EP0Activate                      0x080040f1   Thumb Code    58  usb_core.o(.text)
    USB_OTG_EPActivate                       0x0800412b   Thumb Code   104  usb_core.o(.text)
    USB_OTG_EPDeactivate                     0x08004193   Thumb Code    78  usb_core.o(.text)
    USB_OTG_EPStartXfer                      0x080041e1   Thumb Code   298  usb_core.o(.text)
    USB_OTG_EP0StartXfer                     0x0800430b   Thumb Code   184  usb_core.o(.text)
    USB_OTG_EPSetStall                       0x080043c3   Thumb Code    48  usb_core.o(.text)
    USB_OTG_EPClearStall                     0x080043f3   Thumb Code    50  usb_core.o(.text)
    USB_OTG_ReadDevAllOutEp_itr              0x08004425   Thumb Code    12  usb_core.o(.text)
    USB_OTG_ReadDevOutEP_itr                 0x08004431   Thumb Code    16  usb_core.o(.text)
    USB_OTG_ReadDevAllInEPItr                0x08004441   Thumb Code    12  usb_core.o(.text)
    USB_OTG_EP0_OutStart                     0x0800444d   Thumb Code    32  usb_core.o(.text)
    USB_OTG_ActiveRemoteWakeup               0x0800446d   Thumb Code    66  usb_core.o(.text)
    USB_OTG_UngateClock                      0x080044af   Thumb Code    30  usb_core.o(.text)
    USB_OTG_StopDevice                       0x080044cd   Thumb Code    72  usb_core.o(.text)
    USB_OTG_GetEPStatus                      0x08004515   Thumb Code    66  usb_core.o(.text)
    USB_OTG_SetEPStatus                      0x08004557   Thumb Code   106  usb_core.o(.text)
    DCD_Init                                 0x080045c5   Thumb Code   146  usb_dcd.o(.text)
    DCD_EP_Open                              0x08004657   Thumb Code    60  usb_dcd.o(.text)
    DCD_EP_Close                             0x08004693   Thumb Code    44  usb_dcd.o(.text)
    DCD_EP_PrepareRx                         0x080046bf   Thumb Code    68  usb_dcd.o(.text)
    DCD_EP_Tx                                0x08004703   Thumb Code    62  usb_dcd.o(.text)
    DCD_EP_Stall                             0x08004741   Thumb Code    56  usb_dcd.o(.text)
    DCD_EP_ClrStall                          0x08004779   Thumb Code    56  usb_dcd.o(.text)
    DCD_EP_Flush                             0x080047b1   Thumb Code    24  usb_dcd.o(.text)
    DCD_EP_SetAddress                        0x080047c9   Thumb Code    16  usb_dcd.o(.text)
    DCD_DevConnect                           0x080047d9   Thumb Code    16  usb_dcd.o(.text)
    DCD_DevDisconnect                        0x080047e9   Thumb Code    16  usb_dcd.o(.text)
    DCD_GetEPStatus                          0x080047f9   Thumb Code    38  usb_dcd.o(.text)
    DCD_SetEPStatus                          0x0800481f   Thumb Code    38  usb_dcd.o(.text)
    USBD_OTG_EP1OUT_ISR_Handler              0x08004845   Thumb Code    74  usb_dcd_int.o(.text)
    USBD_OTG_EP1IN_ISR_Handler               0x08004901   Thumb Code   116  usb_dcd_int.o(.text)
    USBD_OTG_ISR_Handler                     0x08004a3b   Thumb Code   324  usb_dcd_int.o(.text)
    USBD_DeInit                              0x08004d9d   Thumb Code     4  usbd_core.o(.text)
    USBD_Init                                0x08004da1   Thumb Code    52  usbd_core.o(.text)
    USBD_SetCfg                              0x08004fad   Thumb Code    26  usbd_core.o(.text)
    USBD_ClrCfg                              0x08004fc7   Thumb Code    14  usbd_core.o(.text)
    USBD_CtlSendData                         0x08004ff5   Thumb Code    32  usbd_ioreq.o(.text)
    USBD_CtlContinueSendData                 0x08005015   Thumb Code    18  usbd_ioreq.o(.text)
    USBD_CtlPrepareRx                        0x08005027   Thumb Code    32  usbd_ioreq.o(.text)
    USBD_CtlContinueRx                       0x08005047   Thumb Code    18  usbd_ioreq.o(.text)
    USBD_CtlSendStatus                       0x08005059   Thumb Code    34  usbd_ioreq.o(.text)
    USBD_CtlReceiveStatus                    0x0800507b   Thumb Code    34  usbd_ioreq.o(.text)
    USBD_GetRxCount                          0x0800509d   Thumb Code    16  usbd_ioreq.o(.text)
    USBD_CtlError                            0x080050ad   Thumb Code    28  usbd_req.o(.text)
    USBD_StdDevReq                           0x08005257   Thumb Code   236  usbd_req.o(.text)
    USBD_StdItfReq                           0x08005343   Thumb Code    54  usbd_req.o(.text)
    USBD_StdEPReq                            0x08005379   Thumb Code   208  usbd_req.o(.text)
    USBD_ParseSetupRequest                   0x08005449   Thumb Code    68  usbd_req.o(.text)
    USBD_GetString                           0x0800548d   Thumb Code    78  usbd_req.o(.text)
    __aeabi_dadd                             0x08005555   Thumb Code   322  dadd.o(.text)
    __aeabi_dsub                             0x08005697   Thumb Code     6  dadd.o(.text)
    __aeabi_drsub                            0x0800569d   Thumb Code     6  dadd.o(.text)
    __aeabi_dmul                             0x080056a3   Thumb Code   228  dmul.o(.text)
    __aeabi_ddiv                             0x08005787   Thumb Code   222  ddiv.o(.text)
    __aeabi_i2d                              0x08005865   Thumb Code    34  dflti.o(.text)
    __aeabi_f2d                              0x08005887   Thumb Code    38  f2d.o(.text)
    __aeabi_d2f                              0x080058ad   Thumb Code    56  d2f.o(.text)
    __aeabi_llsl                             0x080058e5   Thumb Code    30  llshl.o(.text)
    _ll_shift_l                              0x080058e5   Thumb Code     0  llshl.o(.text)
    __aeabi_lasr                             0x08005903   Thumb Code    36  llsshr.o(.text)
    _ll_sshift_r                             0x08005903   Thumb Code     0  llsshr.o(.text)
    __I$use$fp                               0x08005927   Thumb Code     0  iusefp.o(.text)
    _float_round                             0x08005927   Thumb Code    18  fepilogue.o(.text)
    _float_epilogue                          0x08005939   Thumb Code    92  fepilogue.o(.text)
    _double_round                            0x08005995   Thumb Code    30  depilogue.o(.text)
    _double_epilogue                         0x080059b3   Thumb Code   156  depilogue.o(.text)
    _dsqrt                                   0x08005a4f   Thumb Code   162  dsqrt.o(.text)
    __scatterload                            0x08005af1   Thumb Code    28  init.o(.text)
    __scatterload_rt2                        0x08005af1   Thumb Code     0  init.o(.text)
    __aeabi_llsr                             0x08005b15   Thumb Code    32  llushr.o(.text)
    _ll_ushift_r                             0x08005b15   Thumb Code     0  llushr.o(.text)
    __hardfp_sqrt                            0x08005b35   Thumb Code   122  sqrt.o(i.__hardfp_sqrt)
    __scatterload_copy                       0x08005baf   Thumb Code    14  handlers.o(i.__scatterload_copy)
    __scatterload_null                       0x08005bbd   Thumb Code     2  handlers.o(i.__scatterload_null)
    __scatterload_zeroinit                   0x08005bbf   Thumb Code    14  handlers.o(i.__scatterload_zeroinit)
    __set_errno                              0x08005bcd   Thumb Code     6  errno.o(i.__set_errno)
    malloc                                   0x08005bd9   Thumb Code    92  malloc.o(i.malloc)
    FMC_DefaultTimingStruct                  0x08005c44   Data          28  stm32f4xx_fmc.o(.constdata)
    Region$$Table$$Base                      0x08005c60   Number         0  anon$$obj.o(Region$$Table)
    Region$$Table$$Limit                     0x08005c80   Number         0  anon$$obj.o(Region$$Table)
    TM_DELAY_Initialized                     0x20000010   Data           1  tm_stm32f4_delay.o(.data)
    TM_Time                                  0x20000014   Data           4  tm_stm32f4_delay.o(.data)
    TM_Time2                                 0x20000018   Data           4  tm_stm32f4_delay.o(.data)
    mult                                     0x2000001c   Data           4  tm_stm32f4_delay.o(.data)
    TM_INT_DISCO_ButtonPressed               0x20000020   Data           1  tm_stm32f4_disco.o(.data)
    flag_Exp                                 0x20000021   Data           1  stm32f4xx_it.o(.data)
    SystemCoreClock                          0x20000024   Data           4  system_stm32f4xx.o(.data)
    AHBPrescTable                            0x20000028   Data          16  system_stm32f4xx.o(.data)
    tsampling                                0x2000003c   Data           4  paradaconrolada.o(.data)
    vel_max1                                 0x20000040   Data           4  paradaconrolada.o(.data)
    vel_max2                                 0x20000044   Data           4  paradaconrolada.o(.data)
    time                                     0x20000048   Data           4  paradaconrolada.o(.data)
    USBD_DCD_INT_cb                          0x2000004c   Data          44  usbd_core.o(.data)
    USBD_DCD_INT_fops                        0x20000078   Data           4  usbd_core.o(.data)
    SET_TEST_MODE                            0x2000007c   Data           4  usbd_core.o(.data)
    USBD_DeviceQualifierDesc                 0x20000080   Data          10  usbd_desc.o(.data)
    USBD_ep_status                           0x20000090   Data           4  usbd_req.o(.data)
    USBD_default_cfg                         0x20000094   Data           4  usbd_req.o(.data)
    USBD_cfg_status                          0x20000098   Data           4  usbd_req.o(.data)
    __microlib_freelist                      0x2000009c   Data           4  mvars.o(.data)
    __microlib_freelist_initialised          0x200000a0   Data           4  mvars.o(.data)
    encoder1                                 0x200000c0   Data          44  main.o(.bss)
    encoder2                                 0x200000ec   Data          44  main.o(.bss)
    encoder3                                 0x20000118   Data          44  main.o(.bss)
    encoder4                                 0x20000144   Data          44  main.o(.bss)
    TM_INT_USB_VCP_ReceiveBuffer             0x20000170   Data         128  tm_stm32f4_usb_vcp.o(.bss)
    USB_OTG_dev                              0x200001f0   Data        1524  tm_stm32f4_usb_vcp.o(.bss)
    homing                                   0x200007e4   Data           9  homing.o(.bss)
    __heap_base                              0x200007f0   Data           0  startup_stm32f429_439xx.o(HEAP)
    __heap_limit                             0x200009f0   Data           0  startup_stm32f429_439xx.o(HEAP)
    __initial_sp                             0x20000df0   Data           0  startup_stm32f429_439xx.o(STACK)



==============================================================================

Memory Map of the image

  Image Entry point : 0x080001ad

  Load Region LR_IROM1 (Base: 0x08000000, Size: 0x00005d28, Max: 0x00200000, ABSOLUTE)

    Execution Region ER_IROM1 (Base: 0x08000000, Size: 0x00005c80, Max: 0x00200000, ABSOLUTE)

    Base Addr    Size         Type   Attr      Idx    E Section Name        Object

    0x08000000   0x000001ac   Data   RO            3    RESET               startup_stm32f429_439xx.o
    0x080001ac   0x00000000   Code   RO         1310  * .ARM.Collect$$$$00000000  mc_w.l(entry.o)
    0x080001ac   0x00000004   Code   RO         1353    .ARM.Collect$$$$00000001  mc_w.l(entry2.o)
    0x080001b0   0x00000004   Code   RO         1356    .ARM.Collect$$$$00000004  mc_w.l(entry5.o)
    0x080001b4   0x00000000   Code   RO         1358    .ARM.Collect$$$$00000008  mc_w.l(entry7b.o)
    0x080001b4   0x00000000   Code   RO         1360    .ARM.Collect$$$$0000000A  mc_w.l(entry8b.o)
    0x080001b4   0x00000008   Code   RO         1361    .ARM.Collect$$$$0000000B  mc_w.l(entry9a.o)
    0x080001bc   0x00000000   Code   RO         1363    .ARM.Collect$$$$0000000D  mc_w.l(entry10a.o)
    0x080001bc   0x00000000   Code   RO         1365    .ARM.Collect$$$$0000000F  mc_w.l(entry11a.o)
    0x080001bc   0x00000004   Code   RO         1354    .ARM.Collect$$$$00002712  mc_w.l(entry2.o)
    0x080001c0   0x00000024   Code   RO            4    .text               startup_stm32f429_439xx.o
    0x080001e4   0x000000b0   Code   RO           13    .text               misc.o
    0x08000294   0x00000484   Code   RO          151    .text               stm32f4xx_rcc.o
    0x08000718   0x0000020c   Code   RO          177    .text               stm32f4xx_gpio.o
    0x08000924   0x000000e0   Code   RO          225    .text               stm32f4xx_exti.o
    0x08000a04   0x000009dc   Code   RO          249    .text               stm32f4xx_tim.o
    0x080013e0   0x00000154   Code   RO          298    .text               stm32f4xx_dac.o
    0x08001534   0x0000007c   Code   RO          346    .text               stm32f4xx_syscfg.o
    0x080015b0   0x00000758   Code   RO          370    .text               stm32f4xx_fmc.o
    0x08001d08   0x000000a0   Code   RO          397    .text               tm_stm32f4_delay.o
    0x08001da8   0x0000009c   Code   RO          439    .text               tm_stm32f4_disco.o
    0x08001e44   0x0000029c   Code   RO          469    .text               tm_stm32f4_gpio.o
    0x080020e0   0x00000128   Code   RO          558    .text               main.o
    0x08002208   0x00000190   Code   RO          698    .text               stm32f4xx_it.o
    0x08002398   0x00000198   Code   RO          746    .text               system_stm32f4xx.o
    0x08002530   0x00000210   Code   RO          809    .text               tm_stm32f4_sdram.o
    0x08002740   0x000005b8   Code   RO          834    .text               config.o
    0x08002cf8   0x00000b70   Code   RO          861    .text               trapez.o
    0x08003868   0x000000fc   Code   RO          886    .text               functions.o
    0x08003964   0x0000005c   Code   RO          898    .text               controller.o
    0x080039c0   0x00000128   Code   RO          913    .text               paradaconrolada.o
    0x08003ae8   0x00000154   Code   RO          977    .text               usb_bsp.o
    0x08003c3c   0x00000988   Code   RO         1005    .text               usb_core.o
    0x080045c4   0x00000280   Code   RO         1030    .text               usb_dcd.o
    0x08004844   0x00000558   Code   RO         1054    .text               usb_dcd_int.o
    0x08004d9c   0x00000258   Code   RO         1146    .text               usbd_core.o
    0x08004ff4   0x000000b8   Code   RO         1212    .text               usbd_ioreq.o
    0x080050ac   0x000004a8   Code   RO         1236    .text               usbd_req.o
    0x08005554   0x0000014e   Code   RO         1341    .text               mf_w.l(dadd.o)
    0x080056a2   0x000000e4   Code   RO         1343    .text               mf_w.l(dmul.o)
    0x08005786   0x000000de   Code   RO         1345    .text               mf_w.l(ddiv.o)
    0x08005864   0x00000022   Code   RO         1347    .text               mf_w.l(dflti.o)
    0x08005886   0x00000026   Code   RO         1349    .text               mf_w.l(f2d.o)
    0x080058ac   0x00000038   Code   RO         1351    .text               mf_w.l(d2f.o)
    0x080058e4   0x0000001e   Code   RO         1367    .text               mc_w.l(llshl.o)
    0x08005902   0x00000024   Code   RO         1369    .text               mc_w.l(llsshr.o)
    0x08005926   0x00000000   Code   RO         1384    .text               mc_w.l(iusefp.o)
    0x08005926   0x0000006e   Code   RO         1385    .text               mf_w.l(fepilogue.o)
    0x08005994   0x000000ba   Code   RO         1387    .text               mf_w.l(depilogue.o)
    0x08005a4e   0x000000a2   Code   RO         1389    .text               mf_w.l(dsqrt.o)
    0x08005af0   0x00000024   Code   RO         1393    .text               mc_w.l(init.o)
    0x08005b14   0x00000020   Code   RO         1395    .text               mc_w.l(llushr.o)
    0x08005b34   0x0000007a   Code   RO         1298    i.__hardfp_sqrt     m_wm.l(sqrt.o)
    0x08005bae   0x0000000e   Code   RO         1399    i.__scatterload_copy  mc_w.l(handlers.o)
    0x08005bbc   0x00000002   Code   RO         1400    i.__scatterload_null  mc_w.l(handlers.o)
    0x08005bbe   0x0000000e   Code   RO         1401    i.__scatterload_zeroinit  mc_w.l(handlers.o)
    0x08005bcc   0x0000000c   Code   RO         1379    i.__set_errno       mc_w.l(errno.o)
    0x08005bd8   0x0000006c   Code   RO         1314    i.malloc            mc_w.l(malloc.o)
    0x08005c44   0x0000001c   Data   RO          371    .constdata          stm32f4xx_fmc.o
    0x08005c60   0x00000020   Data   RO         1397    Region$$Table       anon$$obj.o


    Execution Region RW_IRAM1 (Base: 0x20000000, Size: 0x00000df0, Max: 0x00030000, ABSOLUTE)

    Base Addr    Size         Type   Attr      Idx    E Section Name        Object

    0x20000000   0x00000010   Data   RW          152    .data               stm32f4xx_rcc.o
    0x20000010   0x00000010   Data   RW          399    .data               tm_stm32f4_delay.o
    0x20000020   0x00000001   Data   RW          440    .data               tm_stm32f4_disco.o
    0x20000021   0x00000001   Data   RW          699    .data               stm32f4xx_it.o
    0x20000022   0x00000002   PAD
    0x20000024   0x00000014   Data   RW          747    .data               system_stm32f4xx.o
    0x20000038   0x00000001   Data   RW          810    .data               tm_stm32f4_sdram.o
    0x20000039   0x00000003   PAD
    0x2000003c   0x00000010   Data   RW          914    .data               paradaconrolada.o
    0x2000004c   0x0000002c   Data   RW         1147    .data               usbd_core.o
    0x20000078   0x00000004   Data   RW         1148    .data               usbd_core.o
    0x2000007c   0x00000004   Data   RW         1149    .data               usbd_core.o
    0x20000080   0x0000000a   Data   RW         1182    .data               usbd_desc.o
    0x2000008a   0x00000002   PAD
    0x2000008c   0x00000010   Data   RW         1238    .data               usbd_req.o
    0x2000009c   0x00000004   Data   RW         1375    .data               mc_w.l(mvars.o)
    0x200000a0   0x00000004   Data   RW         1376    .data               mc_w.l(mvars.o)
    0x200000a4   0x00000004   Data   RW         1380    .data               mc_w.l(errno.o)
    0x200000a8   0x00000016   Zero   RW          470    .bss                tm_stm32f4_gpio.o
    0x200000be   0x00000002   PAD
    0x200000c0   0x000000b0   Zero   RW          562    .bss                main.o
    0x20000170   0x00000674   Zero   RW          777    .bss                tm_stm32f4_usb_vcp.o
    0x200007e4   0x00000009   Zero   RW          944    .bss                homing.o
    0x200007ed   0x00000003   PAD
    0x200007f0   0x00000200   Zero   RW            2    HEAP                startup_stm32f429_439xx.o
    0x200009f0   0x00000400   Zero   RW            1    STACK               startup_stm32f429_439xx.o


==============================================================================

Image component sizes


      Code (inc. data)   RO Data    RW Data    ZI Data      Debug   Object Name

      1464         62          0          0          0       3859   config.o
        92          8          0          0          0       1262   controller.o
       252         40          0          0          0       1941   functions.o
         0          0          0          0          9        553   homing.o
       296         30          0          0        176      52883   main.o
       176         12          0          0          0     312853   misc.o
       296         30          0         16          0       1144   paradaconrolada.o
        36          8        428          0       1536       1064   startup_stm32f429_439xx.o
       340          4          0          0          0       5553   stm32f4xx_dac.o
       224         10          0          0          0       2811   stm32f4xx_exti.o
      1880         30         28          0          0       9078   stm32f4xx_fmc.o
       524         44          0          0          0       4889   stm32f4xx_gpio.o
       400         30          0          1          0       3023   stm32f4xx_it.o
      1156         48          0         16          0      13900   stm32f4xx_rcc.o
       124         16          0          0          0       2065   stm32f4xx_syscfg.o
      2524         52          0          0          0      24414   stm32f4xx_tim.o
       408         36          0         20          0       2071   system_stm32f4xx.o
         0          0          0          0          0       1130   tm_stm32f4_adc.o
       160         16          0         16          0      28642   tm_stm32f4_delay.o
       156         12          0          1          0       1991   tm_stm32f4_disco.o
       668         14          0          0         22       7758   tm_stm32f4_gpio.o
       528         36          0          1          0       1740   tm_stm32f4_sdram.o
         0          0          0          0       1652       1315   tm_stm32f4_usb_vcp.o
      2928         26          0          0          0       6546   trapez.o
       340         10          0          0          0       2383   usb_bsp.o
      2440         16          0          0          0      13766   usb_core.o
       640          0          0          0          0       4408   usb_dcd.o
      1368         22          0          0          0       5790   usb_dcd_int.o
       600          4          0         52          0       5352   usbd_core.o
         0          0          0         10          0       1304   usbd_desc.o
       184          0          0          0          0       2590   usbd_ioreq.o
      1192         42          0         16          0       5709   usbd_req.o

    ----------------------------------------------------------------------
     21396        658        488        156       3400     533787   Object Totals
         0          0         32          0          0          0   (incl. Generated)
         0          0          0          7          5          0   (incl. Padding)

    ----------------------------------------------------------------------

      Code (inc. data)   RO Data    RW Data    ZI Data      Debug   Library Member Name

       122          0          0          0          0        148   sqrt.o
         0          0          0          0          0          0   entry.o
         0          0          0          0          0          0   entry10a.o
         0          0          0          0          0          0   entry11a.o
         8          4          0          0          0          0   entry2.o
         4          0          0          0          0          0   entry5.o
         0          0          0          0          0          0   entry7b.o
         0          0          0          0          0          0   entry8b.o
         8          4          0          0          0          0   entry9a.o
        12          6          0          4          0         68   errno.o
        30          0          0          0          0          0   handlers.o
        36          8          0          0          0         68   init.o
         0          0          0          0          0          0   iusefp.o
        30          0          0          0          0         68   llshl.o
        36          0          0          0          0         68   llsshr.o
        32          0          0          0          0         68   llushr.o
       108         16          0          0          0         84   malloc.o
         0          0          0          8          0          0   mvars.o
        56          0          0          0          0         88   d2f.o
       334          0          0          0          0        148   dadd.o
       222          0          0          0          0        100   ddiv.o
       186          0          0          0          0        176   depilogue.o
        34          0          0          0          0         76   dflti.o
       228          0          0          0          0         96   dmul.o
       162          0          0          0          0        100   dsqrt.o
        38          0          0          0          0         68   f2d.o
       110          0          0          0          0        168   fepilogue.o

    ----------------------------------------------------------------------
      1796         38          0         12          0       1592   Library Totals
         0          0          0          0          0          0   (incl. Padding)

    ----------------------------------------------------------------------

      Code (inc. data)   RO Data    RW Data    ZI Data      Debug   Library Name

       122          0          0          0          0        148   m_wm.l
       304         38          0         12          0        424   mc_w.l
      1370          0          0          0          0       1020   mf_w.l

    ----------------------------------------------------------------------
      1796         38          0         12          0       1592   Library Totals

    ----------------------------------------------------------------------

==============================================================================


      Code (inc. data)   RO Data    RW Data    ZI Data      Debug   

     23192        696        488        168       3400     528859   Grand Totals
     23192        696        488        168       3400     528859   ELF Image Totals
     23192        696        488        168          0          0   ROM Totals

==============================================================================

    Total RO  Size (Code + RO Data)                23680 (  23.13kB)
    Total RW  Size (RW Data + ZI Data)              3568 (   3.48kB)
    Total ROM Size (Code + RO Data + RW Data)      23848 (  23.29kB)

==============================================================================

